:0200000480007A
:10000000B72F0000938F0F8073900F306F00400365
:100010001300000013000000130000001300000094
:100020001300000013000000130000001300000084
:100030001300000013000000130000001300000074
:100040009702000093824211739052309300000097
:10005000130100009301000013020000930200004E
:100060001303000093030000130400009304000036
:10007000130500009305000013060000930600001E
:100080001307000093070000130800009308000006
:100090001309000093090000130A0000930A0000EE
:1000A000130B0000930B0000130C0000930C0000D6
:1000B000130D0000930D0000130E0000930E0000BE
:1000C000130F0000930F000097110200938141B0BD
:1000D0001705020013050533979503009385056EF8
:1000E00013060000EF00001A170502001305452D46
:1000F000970502009385852D13060000EF008018F8
:1001000017A503001305C56B97B503009385056B11
:1001100037B6ABAB1306B6BAEF00C01617B1030083
:100120001301016AEF7010699392120093D21200CA
:100130009382D2FF638A02008322010013014100EF
:100140006F0000177300203083220100130141006B
:10015000730020301301C1FF23205100F32220340B
:10016000E3C402FC8322010013014100130141F8A2
:1001700023221100232421002326310023284100BB
:10018000232A5100232C6100232E71002320810299
:10019000232291022324A1022326B1022328C10293
:1001A000232AD102232CE102232EF1022320010570
:1001B0002322110523242105232631052328410567
:1001C000232A5105232C6105232E71052320810745
:1001D000232291072324A1072326B1072328C1073F
:1001E000232AD107232CE107232EF107732520347E
:1001F000F3251034130601006F000000731015344E
:1002000083204100032181008321C10003220101D9
:1002100083224101032381018323C10103240102BD
:1002200083244102032581028325C10203260103A1
:1002300083264103032781038327C1030328010485
:1002400083284104032981048329C104032A010569
:10025000832A4105032B8105832BC105032C01064D
:10026000832C4106032D8106832DC106032E010731
:10027000832E4107032F8107832FC1071301C10775
:10028000730020302320C5006376B50013054500B8
:100290006FF05FFF678000000000000000000000BA
:1002A000000000000000000000000000000000004E
:1002B000130101F8232011002322210023243100FF
:1002C0002326410023285100232A6100232C71009A
:1002D000232E8100232091022322A1022324B10294
:1002E0002326C1022328D102232AE102232CF10272
:1002F000232E010323201105232221052324310568
:100300002326410523285105232A6105232C710545
:10031000232E8105232091072322A1072324B1073F
:100320002326C1072328D107232AE107232CF1071D
:100330009702020083A2020923A02200F3221034B4
:10034000232E5106EF00804617010200032181078A
:10035000032101008322C10773901234B7220000E9
:100360009382028873A00230832001000322C1001F
:100370008322010103234101832381010324C1015D
:100380008324010203254102832581020326C10241
:100390008326010303274103832781030328C10325
:1003A000832801040329410483298104032AC10409
:1003B000832A0105032B4105832B8105032CC105ED
:1003C000832C0106032D4106832D8106032EC106D1
:1003D000832E0107032F4107832F81071301010893
:1003E00073002030970202009382C20123A0120002
:1003F00023A2220023A4320023A6420023A85200F5
:1004000023AA620023AC720023AE820023A09202D2
:1004100023A2A20223A4B20223A6C20223A8D202CC
:1004200023AAE20223ACF20223AE020323A01205A8
:1004300023A2220523A4320523A6420523A85205A0
:1004400023AA620523AC720523AE820523A092077E
:1004500023A2A20723A4B20723A6C20723A8D20778
:1004600023AAE20723ACF207EF7010231701020062
:10047000032141F5032101008322C1077390123447
:10048000B72200009382028873A00230832001000B
:100490000322C1008322010103234101832381013F
:1004A0000324C10183240102032541028325810223
:1004B0000326C10283260103032741038327810307
:1004C0000328C103832801040329410483298104EB
:1004D000032AC104832A0105032B4105832B8105CF
:1004E000032CC105832C0106032D4106832D8106B3
:1004F000032EC106832E0107032F4107832F810797
:10050000130101087300203097020200938282EFEA
:1005100083A0020003A1420083A1820003A2C200C3
:1005200083A2020103A3420183A3820103A4C201A7
:1005300083A4020203A5420283A5820203A6C2028B
:1005400083A6020303A7420383A7820303A8C2036F
:1005500083A8020403A9420483A9820403AAC20453
:1005600083AA020503AB420583AB820503ACC20537
:1005700083AC020603AD420683AD820603AEC2061B
:1005800083AE020703AFC20983AF82076780000012
:1005900073700430130101F823201100232221007D
:1005A000232431002326410023285100232A6100FF
:1005B000232C7100232E8100232091022322A102EB
:1005C0002324B1022326C1022328D102232AE102D7
:1005D000232CF102232E01032320110523222105C0
:1005E000232431052326410523285105232A6105AB
:1005F000232C7105232E8105232091072322A10797
:100600002324B1072326C1072328D107232AE10782
:10061000232CF1079702020083A2C2DA23A0220052
:10062000232E1106EF30D00817010200032181D9D3
:10063000032101008322C10773901234B722000006
:100640009382028873A00230832001000322C1003C
:100650008322010103234101832381010324C1017A
:100660008324010203254102832581020326C1025E
:100670008326010303274103832781030328C10342
:10068000832801040329410483298104032AC10426
:10069000832A0105032B4105832B8105032CC1050A
:1006A000832C0106032D4106832D8106032EC106EE
:1006B000832E0107032F4107832F810713010108B0
:1006C0007300203097070200938787D003A70700A5
:1006D0009307F0FF6306F700737004306F000000AB
:1006E000737004306F000000130101FF2326A10086
:1006F0008327C100739047301300000013010101EC
:1007000067800000130101FFF32740302326F1002A
:1007100073F043308327C1001385070013010101E3
:1007200067800000130101FF2326A1002324B100EC
:100730002322C1008327C1009387C7FF2326F1002E
:10074000032781008327C10023A0E7008327C1007E
:10075000938787FA2326F100032741008327C100EE
:1007600023A0E7008327C100938787FE2326F1009B
:1007700093870100138707008327C10023A0E700A8
:100780008327C100938747FF2326F1001707000046
:10079000130787F38327C10023A0E7008327C10045
:1007A000138507001301010167800000130101FF99
:1007B00023261100EF70C063EF3000469307050059
:1007C00063840700EF30C06E130000008320C10077
:1007D0001301010167800000130101FD23261102AE
:1007E0002326A1002324B1002322C1001305800386
:1007F000EF60C05A232CA100832781016382071276
:10080000970702009387C7BB83A70700639C070075
:10081000970702009387C7BA0327810123A0E70047
:10082000EF00405E032781009307100063F6E700A6
:10083000930710002324F10083278101239A0702E4
:10084000832781010327810023A6E70283278101F3
:100850000327410023A8E702832781010327C10062
:1008600023A0E700832781019387470013850700B2
:10087000EF00C071832781019387870113850700EB
:10088000EF00C070832781010327810123A8E700BF
:10089000832781010327810123A2E7021307200098
:1008A000832781003307F7408327810123ACE700CA
:1008B0008327810103A7C70297070200938707C315
:1008C00083A7070063FCE7008327810103A7C70212
:1008D00097070200938787C123A0E7008327810140
:1008E00003A7C7029307070093972700B387E70082
:1008F0009397270017070200130787B83387E7008D
:10090000832781019387470093850700130507001C
:10091000EF00806993071000232EF1006F00C000E4
:100920009307F0FF232EF1008327C10113850700F1
:100930008320C1021301010367800000130101FD40
:10094000232611022326A1002324B10097070200C9
:10095000938707BA83A707000327C100B307F700EF
:10096000232EF10097070200938787A583A707002E
:100970009387470013850700EF0040779707020031
:10098000938707A483A707000327C10123A2E700D9
:10099000970702009387C7B583A707000327C10104
:1009A0006378F702970702009387C7B203A707008F
:1009B000970702009387C7A083A707009387470084
:1009C0009385070013050700EF00C0656F00C002A4
:1009D000970702009387C7AF03A707009707020096
:1009E0009387079E83A70700938747009385070097
:1009F00013050700EF00006383278100638007026F
:100A0000970702009387C79B83A7070093878701F7
:100A10009385070003258100EF00C06013000000EC
:100A20008320C1021301010367800000130101FE4E
:100A3000232E11006F00400A7370043097070200E4
:100A4000938787A983A7C70083A7C7002326F10040
:100A50008327C1009387870113850700EF00006992
:100A6000736004308327C100938747001385070014
:100A7000EF00C0678327C10003A7C70297070200E2
:100A80009387C7A683A7070063FCE7008327C100FD
:100A900003A7C70297070200938747A523A0E70093
:100AA0008327C10003A7C702930707009397270076
:100AB000B387E70093972700170702001307479CA7
:100AC0003387E7008327C10093874700938507009A
:100AD00013050700EF00404D970702009387C79F5B
:100AE00083A70700E39A07F4130000008320C101E5
:100AF0001301010267800000130101FE232E110083
:100B0000EF20906E13070500970702009387879EDA
:100B100083A707003307F740970702009387C79D15
:100B200023A0E7006F008016970702009387479C79
:100B300083A7070013871700970702009387479B37
:100B400023A0E700970702009387079B83A707006E
:100B50001387F7FF970702009387079A23A0E70000
:100B6000970702009387C79883A70700639607102B
:100B7000970702009387C79583A707002326F100F4
:100B8000970702009387079503A7070097070200BE
:100B90009387079423A0E700970702009387879322
:100BA0000327C10023A0E7006F00000D9707020094
:100BB0009387079283A7070083A7C70083A7C7006F
:100BC0002324F1008327810003A747009707020031
:100BD0009387079283A7070063F4E7006F00000B79
:100BE00073700430832781009387470013850700C3
:100BF000EF00C04F8327810083A78702638A070025
:100C0000832781009387870113850700EF00004E3B
:100C1000736004308327810003A7C702970702008F
:100C20009387C78C83A7070063FCE70083278100B5
:100C300003A7C702970702009387478B23A0E7000B
:100C40008327810003A7C702930707009397270014
:100C5000B387E7009397270017070200130747821F
:100C60003387E70083278100938747009385070038
:100C700013050700EF00403397070200938747856D
:100C800083A7070083A70700E39207F297070200F4
:100C90009387878683A70700E39807E897070200F2
:100CA0009387078503A70700970702009387878428
:100CB00023A0E700130000008320C10113010102FB
:100CC00067800000130101FE232E1100EFF01FD6F4
:100CD000EFF09FE26F000003970702009387078100
:100CE00083A7070063880710970702009387078090
:100CF00083A707001387F7FF97F701009387077F04
:100D000023A0E70097F701009387477E03A707001A
:100D100097F601009386C6769307070093972700FE
:100D2000B387E70093972700B387F60083A70700F0
:100D3000E38407FA97F701009387477B03A707002F
:100D40009307070093972700B387E700939727003F
:100D500017F701001307C772B387E7002326F100D6
:100D60008327C10083A7470003A747008327C1004B
:100D700023A2E7008327C10003A747008327C10000
:100D800093878700631CF7008327C10083A7470070
:100D900003A747008327C10023A2E7008327C100E0
:100DA00083A7470003A7C70097F701009387476110
:100DB00023A0E70097F701009387876083A70700C8
:100DC00083A6070097F701009387875F03A70700B3
:100DD00097F701009387C75E83A7070083A70703E0
:100DE0009385070013050700E78006001300000045
:100DF0006F008000130000008320C1011301010275
:100E000067800000130101FE232E1100232601003C
:100E10006F0080030327C100930707009397270003
:100E2000B387E7009397270017F70100130747657B
:100E3000B387E70013850700EF00C00F8327C100C9
:100E4000938717002326F1000327C10093071000A2
:100E5000E3F2E7FC17F5010013050565EF00800DCF
:100E600017F5010013058565EF00C00C17F50100AB
:100E700013058566EF00000C97F70100938747651F
:100E800017F701001307476223A0E70097F7010057
:100E90009387476417F701001307476223A0E70011
:100EA000130000008320C1011301010267800000CC
:100EB000130101FD232611022326A1008327C1006F
:100EC00083A7C70083A7C700232CF10083278101D4
:100ED0009387870113850700EF0040218327810155
:100EE000938787019385070017F501001305C55EF9
:100EF000EF00800B8327810103A7C70297F701004A
:100F00009387074C83A7070083A7C7026368F7008E
:100F100093071000232EF1006F008000232E0100A4
:100F20008327C101138507008320C1021301010338
:100F300067800000130101FF2326A1008327C10061
:100F4000138787008327C10023A2E7008327C100FE
:100F50001307F0FF23A4E7008327C100138787004E
:100F60008327C10023A6E7008327C10013878700DA
:100F70008327C10023A8E7008327C10023A007001F
:100F8000130000001301010167800000130101FF3D
:100F90002326A1008327C10023A807001300000017
:100FA0001301010167800000130101FE2326A10047
:100FB0002324B1008327C10083A74700232EF1001B
:100FC000832781000327C10123A2E7008327C101F2
:100FD00003A787008327810023A4E7008327C1019B
:100FE00083A787000327810023A2E7008327C1018D
:100FF0000327810023A4E700832781000327C10082
:1010000023A8E7008327C10083A7070013871700E1
:101010008327C10023A0E700130000001301010291
:1010200067800000130101FE2326A1002324B100E4
:101030008327810083A70700232CF1000327810168
:101040009307F0FF631AF7008327C10083A7070106
:10105000232EF1006F0040038327C1009387870090
:10106000232EF1006F0000018327C10183A74700F1
:10107000232EF1008327C10183A7470083A7070020
:1010800003278101E372F7FE8327C10103A747000D
:101090008327810023A2E7008327810083A74700DD
:1010A0000327810023A4E700832781000327C101D0
:1010B00023A4E7008327C1010327810023A2E700BF
:1010C000832781000327C10023A8E7008327C100ED
:1010D00083A70700138717008327C10023A0E70019
:1010E000130000001301010267800000130101FEDC
:1010F0002326A1008327C10083A70701232EF10027
:101100008327C10083A747000327C1000327870067
:1011100023A4E7008327C10083A787000327C1001A
:101120000327470023A2E7008327C10183A74700C5
:101130000327C100631AF7008327C10003A78700B4
:101140008327C10123A2E7008327C10023A807004A
:101150008327C10183A707001387F7FF8327C101F6
:1011600023A0E7008327C10183A707001385070099
:101170001301010267800000130101FD2326110203
:10118000232481022326A1002324B1008327C10048
:10119000232EF1008327C10163960700737004308A
:1011A0006F000000EF30507B8327C10103A40700CC
:1011B0008327C10103A7C7038327C10183A70704AE
:1011C0009385070013050700EF7010709307050063
:1011D0003307F4008327C10123A2E7008327C1015D
:1011E00023AC07028327C10103A707008327C1019E
:1011F00023A4E7008327C10103A407008327C101BB
:1012000083A7C7031387F7FF8327C10183A70704B9
:101210009385070013050700EF70106B9307050017
:101220003307F4008327C10123A6E7008327C10108
:101230001307F0FF23A2E7048327C1011307F0FF80
:1012400023A4E70483278100639A07028327C1014F
:1012500083A70701638407048327C10193870701DC
:1012600013850700EF308006130705009307100071
:101270006316F702EFF0CFB16F0040028327C10180
:101280009387070113850700EFF0DFCA8327C101A9
:101290009387470213850700EFF0DFC9EF30D06F67
:1012A00093071000138507008320C10203248102E5
:1012B0001301010367800000130101FD23261102C1
:1012C0002326A1002324B10093070600A303F10005
:1012D000232C01008327C10063960700737004303C
:1012E0006F0000008327810063960700232E010012
:1012F0006F00C001832581000325C100EF70D05C21
:101300009307050093871700232EF1008327C1015F
:101310009387470513850700EF505028232AA10023
:10132000832741016382070683278100639A0700B0
:10133000832741010327410123A0E7006F004001FB
:1013400083274101138747058327410123A0E70035
:10135000832741010327C10023AEE7028327410110
:101360000327810023A0E704930510000325410112
:10137000EFF09FE083274101034771002388E704D2
:1013800083274101232CF100832781016396070005
:10139000737004306F0000008327810113850700FC
:1013A0008320C1021301010367800000130101FDC6
:1013B0002326110293070500A307F100130540053A
:1013C000EF50D01D232EA1008327C101638C070895
:1013D0008327C10123A207008327C10123A007009F
:1013E0008327C10123A407008327C10123A6070087
:1013F0008327C10123AC07028327C1011307100013
:1014000023AEE7028327C10123A007048327C1017C
:101410001307F0FF23A2E7048327C1011307F0FF9E
:1014200023A4E7048327C1010347F1002388E704CD
:101430008327C1019387070113850700EFF09FAF52
:101440008327C1019387470213850700EFF09FAE02
:101450009306000013060000930500000325C10158
:10146000EF00001E8327C101138507008320C102FE
:101470001301010367800000130101FD23261102FF
:10148000232481022326A1008327C100232CF100FD
:101490008327810163960700737004306F0000009A
:1014A0008327810103A44700EF30501A93070500FA
:1014B0006312F4048327810183A7C7001387F7FF12
:1014C0008327810123A6E7008327810183A7C70023
:1014D000639C0700930600001306000093050000BC
:1014E00003258101EF00C01593071000232EF100A2
:1014F0006F008000232E01008327C10113850700A0
:101500008320C102032481021301010367800000CC
:10151000130101FD23261102232481022326A100A9
:101520002324B1008327C100232CF10083278101EC
:1015300063960700737004306F00000083278101F9
:1015400003A44700EF309010930705006312F402E4
:101550008327810183A7C700138717008327810191
:1015600023A6E70093071000232EF1006F00C003AD
:1015700093060000032681009305000003258101E6
:10158000EF00C058232EA1000327C10193071000CC
:10159000631CF7008327810183A7C7001387170007
:1015A0008327810123A6E7008327C1011385070054
:1015B0008320C1020324810213010103678000001C
:1015C000130101FD232611022326A1002324B100CB
:1015D0008327C10063960700737004306F0000001A
:1015E000032781008327C10063F6E700737004308E
:1015F0006F00000013062000930500000325C100C2
:10160000EFF09FCB232EA1008327C1016388070041
:101610008327C1010327810023ACE7028327C1018F
:1016200063960700737004306F0000008327C101C8
:10163000138507008320C1021301010367800000A6
:10164000130101FC232E11022326A1002324B10043
:101650002322C1002320D100232601028327C100B9
:101660002324F102832781026396070073700430FC
:101670006F000000832781006398070083278102A1
:1016800083A7070463960700930710006F0080008C
:101690009307000063960700737004306F0000002A
:1016A0000327010093072000631AF70083278102B4
:1016B00003A7C703930710006316F70093071000F2
:1016C0006F0080009307000063960700737004307A
:1016D0006F000000EF30C0799307050063960700A4
:1016E0008327410063960700930710006F00800076
:1016F0009307000063960700737004306F000000CA
:10170000EF3090258327810203A787038327810277
:1017100083A7C7036368F70003270100930720002E
:101720006310F7060326010083258100032581024B
:10173000EF00101C2322A1028327810283A7470206
:10174000638407028327810293874702138507007A
:10175000EF20D0371307050093071000631CF70034
:10176000EFE01FE36F00000183274102638407005D
:10177000EFE01FE2EF305022930710006F00400FA0
:101780008327410063980700EF3010219307000082
:101790006F00000E8327C102639C07009307C101FD
:1017A00013850700EF209057930710002326F102BE
:1017B000EF30901EEF200004EF30101A83278102D3
:1017C00003A747049307F0FF6316F70083278102FE
:1017D00023A207048327810203A787049307F0FF4E
:1017E0006316F7008327810223A40704EF30D01A81
:1017F000130741009307C1019305070013850700F4
:10180000EF20905693070500639C0704032581028F
:10181000EF00504693070500638C0702832781027F
:1018200093870701032741009305070013850700ED
:10183000EF20500403258102EF00902CEF10D07DA3
:1018400093070500E39E07EAEFE09FD46FF05FEB9C
:1018500003258102EF00D02AEF10107C6FF05FEAC1
:1018600003258102EF00D029EF10107B93070000C1
:10187000138507008320C103130101046780000062
:10188000130101FD232611022326A1002324B10008
:101890002322C1002320D1008327C100232CF10083
:1018A0008327810163960700737004306F00000086
:1018B00083278100639807008327810183A707049A
:1018C00063960700930710006F00800093070000E5
:1018D00063960700737004306F0000000327010057
:1018E00093072000631AF7008327810103A7C7032A
:1018F000930710006316F700930710006F00800035
:101900009307000063960700737004306F000000B7
:10191000EFE05FDF93070500232AF10083278101B1
:1019200003A787038327810183A7C7036368F700A1
:1019300003270100930720006310F7080326010026
:101940008325810003258101EF00807A83278101AF
:1019500003A787049307F0FF6310F704832781012F
:1019600083A7470263840704832781019387470283
:1019700013850700EF209015930705006388070281
:101980008327410063840702832741001307100067
:1019900023A0E7006F0080018327810183A78704CC
:1019A000138717008327810123A4E70493071000FE
:1019B000232EF1006F008000232E010083274101B8
:1019C00013850700EFE05FD28327C101138507006D
:1019D0008320C1021301010367800000130101FD90
:1019E000232611022326A1002324B1008327C1004E
:1019F000232CF10083278101639607007370043064
:101A00006F0000008327810183A707046386070016
:101A1000737004306F0000008327810183A70700E3
:101A2000639807008327810183A747006396070017
:101A3000930710006F008000930700006396070073
:101A4000737004306F000000EFE0DFCB93070500F8
:101A5000232AF1008327810103A7870383278101BC
:101A600083A7C7036372F7088327810183A78703CE
:101A7000138717008327810123ACE70283278101A5
:101A800003A787049307F0FF6310F70483278101FE
:101A900083A7470263840704832781019387470252
:101AA00013850700EF209002930705006388070263
:101AB00083278100638407028327810013071000B6
:101AC00023A0E7006F0080018327810183A787049B
:101AD000138717008327810123A4E70493071000CD
:101AE000232EF1006F008000232E01008327410187
:101AF00013850700EFE05FBF8327C101138507004F
:101B00008320C1021301010367800000130101FC5F
:101B1000232E11022326A1002324B1002322C10079
:101B20002320D100232601028327C1002324F102B0
:101B30008327810263960700737004306F000000F2
:101B400083278100639807008327810283A7070406
:101B500063960700930710006F0080009307000052
:101B600063960700737004306F000000EF30403060
:101B700093070500639607008327410063960700DB
:101B8000930710006F008000930700006396070022
:101B9000737004306F000000EF30005C8327810217
:101BA00083A787036382070C8327810283A7C7006B
:101BB0002322F1028325810003258102EF00806B3F
:101BC00083270100639207068327810283A7870387
:101BD0001387F7FF8327810223ACE7028327810263
:101BE00083A70700639A0700EF30C065130705005D
:101BF0008327810223A2E7008327810283A70701AD
:101C0000638E0704832781029387070113850700EA
:101C1000EF20C06B13070500930710006310F70453
:101C2000EFE01F976F0080038327810203274102A3
:101C300023A6E7008327810283A747026380070268
:101C4000832781029387470213850700EF200068EE
:101C50009307050063840700EFE09F93EF30C053C4
:101C6000930710006F0080118327410063980700DD
:101C7000EF308052930700006F0040108327C102AD
:101C8000639C07009307C10113850700EF2010092B
:101C9000930710002326F102EF300050EF1090352B
:101CA000EF30804B8327810203A747049307F0FF9F
:101CB0006316F7008327810223A20704832781028A
:101CC00003A787049307F0FF6316F70083278102B9
:101CD00023A40704EF30404C130741009307C101D0
:101CE0009305070013850700EF20100893070500F0
:101CF000639E070603258102EF00406F93070500EE
:101D0000638E07048327810283A70700639E070071
:101D1000EF3080448327810283A7470013850700A3
:101D2000EF30001AEF304047832781029387470244
:101D3000032741009305070013850700EF20803338
:101D400003258102EF00C05BEF10102D9307050003
:101D5000E39407E4EFE0DF836FF01FE403258102E3
:101D6000EF00005AEF10502B6FF01FE303258102A4
:101D7000EF000059EF10502A930700001385070069
:101D80008320C1031301010467800000130101FDDA
:101D9000232611022326A1002324B1002322C100FF
:101DA0008327C100232CF10083278101639607005C
:101DB000737004306F000000832781006398070070
:101DC0008327810183A70704639607009307100008
:101DD0006F00800093070000639607007370043063
:101DE0006F000000EFE01F9293070500232AF10027
:101DF0008327810183A787036388070883258100E0
:101E000003258101EF0000478327810183A7870312
:101E10001387F7FF8327810123ACE7028327810122
:101E200003A747049307F0FF6310F704832781019A
:101E300083A7070163840704832781019387070130
:101E400013850700EF208048930705006388070289
:101E50008327410063840702832741001307100092
:101E600023A0E7006F0080018327810183A7470437
:101E7000138717008327810123A2E704930710002B
:101E8000232EF1006F008000232E010083274101E3
:101E900013850700EFE05F858327C10113850700E5
:101EA0008320C1021301010367800000130101FDBB
:101EB000232611022326A1002324B1008327C10079
:101EC000232CF1008327810163960700737004308F
:101ED0006F0000008327810063980700832781013A
:101EE00083A7070463960700930710006F00800024
:101EF0009307000063960700737004306F000000C2
:101F00008327810183A70704639607007370043059
:101F10006F000000EFE00FFF93070500232AF10098
:101F20008327810183A78703638A070283278101AF
:101F300083A7C7002328F1008325810003258101A1
:101F4000EF004033832781010327010123A6E70027
:101F500093071000232EF1006F008000232E010054
:101F60008327410113850700EFE00FF88327C101A4
:101F7000138507008320C10213010103678000005D
:101F8000130101FD232611022326A1008327C1008E
:101F900063960700737004306F000000EF30C01BC1
:101FA0008327C10083A78703232EF100EF30C01ED3
:101FB0008327C101138507008320C1021301010398
:101FC00067800000130101FD232611022326A100D2
:101FD0008327C100232EF1008327C10163960700E8
:101FE000737004306F000000EF3000178327C101C9
:101FF00003A7C7038327C10183A78703B307F7405C
:10200000232CF100EF30401983278101138507004D
:102010008320C1021301010367800000130101FE48
:102020002326A1008327C100639607007370043044
:102030006F0000008327C10083A78703232EF100D0
:102040008327C10113850700130101026780000087
:10205000130101FD232611022326A1008327C100BD
:10206000232EF1008327C1016396070073700430AB
:102070006F0000000325C101EF00900C0325C10192
:10208000EF409071130000008320C102130101038F
:1020900067800000130101FF2326A1008327C100F0
:1020A00083A7C7041385070013010101678000009F
:1020B000130101FF2326A1002324B1008327C100BF
:1020C0000327810023A6E704130000001301010188
:1020D00067800000130101FF2326A1008327C100B0
:1020E00083C70705138507001301010167800000FE
:1020F000130101FD232611022326A1002324B10090
:102100002322C100232E01008327C10083A70704D7
:10211000639807028327C10083A70700639807120B
:102120008327C10083A7470013850700EF20106FA6
:10213000232EA1008327C10023A207006F000011F6
:1021400083274100639407068327C10003A7870004
:102150008327C10083A70704138607008325810016
:1021600013050700EF40107A8327C10003A78700FB
:102170008327C10083A707043307F7008327C10023
:1021800023A4E7008327C10003A787008327C1009A
:1021900083A74700636CF70A8327C10003A70700E2
:1021A0008327C10023A4E7006F00400A8327C100F2
:1021B00003A7C7008327C10083A70704138607006E
:1021C0008325810013050700EF40D0738327C100EA
:1021D00003A7C7008327C10083A70704B307F04004
:1021E0003307F7008327C10023A6E7008327C10038
:1021F00003A7C7008327C10083A707006372F70204
:102200008327C10003A747008327C10083A70704D2
:10221000B307F0403307F7008327C10023A6E70088
:1022200003274100930720006312F7028327C100B0
:1022300083A78703638C07008327C10083A78703D5
:102240001387F7FF8327C10023ACE7028327C10070
:1022500083A78703138717008327C10023ACE702F6
:102260008327C101138507008320C10213010103E5
:1022700067800000130101FE232E11002326A10018
:102280002324B1008327C10083A7070463820706C4
:102290008327C10003A7C7008327C10083A70704C2
:1022A0003307F7008327C10023A6E7008327C10077
:1022B00003A7C7008327C10083A74700636AF7000D
:1022C0008327C10003A707008327C10023A6E700D7
:1022D0008327C10003A7C7008327C10083A7070482
:1022E000138607009305070003258100EF409061E6
:1022F000130000008320C101130101026780000068
:10230000130101FE232E11002326A100EF20D0642B
:102310006F0000048327C10083A74702638207047C
:102320008327C1009387470213850700EF10107AB7
:102330009307050063840700EF2000338327C10063
:1023400083A787041387F7FF8327C10023A4E7042B
:102350008327C10083A78704E34EF0FA6F00800053
:10236000130000008327C1001307F0FF23A4E70434
:10237000EF209062EF20505E6F0000048327C100C1
:1023800083A70701638207048327C100938707019E
:1023900013850700EF10907393070500638407000F
:1023A000EF20802C8327C10083A747041387F7FF02
:1023B0008327C10023A2E7048327C10083A7470422
:1023C000E34EF0FA6F008000130000008327C10085
:1023D0001307F0FF23A2E704EF20105C13000000B6
:1023E0008320C1011301010267800000130101FD78
:1023F000232611022326A100EF2010568327C100B7
:1024000083A787036398070093071000232EF1002A
:102410006F008000232E0100EF2010588327C10198
:10242000138507008320C1021301010367800000A8
:10243000130101FE2326A1008327C1006396070034
:10244000737004306F0000008327C10083A78703E7
:102450006398070093071000232EF1006F0080009F
:10246000232E01008327C1011385070013010102F8
:1024700067800000130101FD232611022326A1001D
:10248000EF20904D8327C10003A787038327C10056
:1024900083A7C7036318F70093071000232EF100EA
:1024A0006F008000232E0100EF20104F8327C10111
:1024B000138507008320C102130101036780000018
:1024C000130101FE2326A1008327C10063960700A4
:1024D000737004306F0000008327C10003A78703D7
:1024E0008327C10083A7C7036318F7009307100071
:1024F000232EF1006F008000232E01008327C101ED
:10250000138507001301010267800000130101FD1C
:10251000232611022326A1002324B1002322C10077
:102520008327C100232CF10073700430032581013F
:10253000EFF05FF493070500638C070283274100E7
:102540006382070283278101938707019385070030
:1025500003254100EFE08FBE736004309307C0FF96
:102560006F00000873600430930700006F0040079D
:1025700073600430737004308327810103A78703DD
:102580008327810183A7C7036376F704130600003E
:102590008325810003258101EFF09FB5930710008B
:1025A000232EF1008327810183A747026386070258
:1025B000832781019387470213850700EFE05F8F30
:1025C00093070500638A07009307B0FF232EF100ED
:1025D0006F008000232E0100736004308327C10147
:1025E000138507008320C1021301010367800000E7
:1025F000130101FD232611022326A1002324B1008B
:102600002322C1008327C100232CF1007370043002
:102610008327810183A78703639C070283274100E7
:10262000638207028327810193874702938507000E
:1026300003254100EFE08FB0736004309307C0FFC3
:102640006F00C00D73600430930700006F00000D31
:1026500073600430737004308327810183A787037C
:102660006388070A8327810103A7C70083278101A5
:1026700083A707043307F7008327810123A6E70018
:102680008327810103A7C7008327810183A7470010
:10269000636AF7008327810103A70700832781016D
:1026A00023A6E7008327810183A787031387F7FF0A
:1026B0008327810123ACE7028327810103A7C70099
:1026C0008327810183A7070413860700930507006A
:1026D00003258100EF40102393071000232EF10003
:1026E0008327810183A7070163860702832781016E
:1026F0009387070113850700EFE08FFB9307050021
:10270000638A07009307B0FF232EF1006F0080005B
:10271000232E0100736004308327C1011385070055
:102720008320C1021301010367800000130101FD32
:10273000232611022326A1002324B1002322C10055
:102740008327C100232EF1008327C10103A787033C
:102750008327C10183A7C7036374F704130600002E
:10276000832581000325C101EFF09F988327410055
:10277000639807028327C10183A747026382070288
:102780008327C1019387470213850700EFE04FF2CB
:102790009307050063860700930710006F00800011
:1027A00083274100138507008320C1021301010321
:1027B00067800000130101FD232611022326A100DA
:1027C0002324B1002322C1008327C100232CF10060
:1027D0008327810183A787036380070C83278101F7
:1027E00003A7C7008327810183A707043307F700E6
:1027F0008327810123A6E7008327810103A7C70060
:102800008327810183A74700636AF700832781013B
:1028100003A707008327810123A6E70083278101FF
:1028200083A787031387F7FF8327810123ACE70280
:102830008327810103A7C7008327810183A707049A
:10284000138607009305070003258100EF40900BD6
:102850008327410083A70700639A0702832781012A
:1028600083A70701638407028327810193870701F8
:1028700013850700EFE0CFE39307050063880700A7
:10288000832741001307100023A0E70093071000DF
:10289000232EF1006F008000232E01008327C10149
:1028A000138507008320C102130101036780000024
:1028B000130101FE2326A1002324B100232E0100D1
:1028C0006F00800617770300130787EB8327C1018A
:1028D00093973700B307F70083A7070063900704B7
:1028E000177703001307C7E98327C10193973700C0
:1028F000B307F7000327810023A0E7001777030041
:10290000130707E88327C10193973700B307F70040
:102910000327C10023A2E7006F00C0018327C10184
:1029200093871700232EF1000327C101930770003E
:10293000E3FAE7F8130000001301010267800000CA
:10294000130101FE2326A100232E01006F00C00405
:10295000177703001307C7E28327C1019397370056
:10296000B307F70083A747000327C1006310F702EE
:10297000177703001307C7E08327C1019397370038
:10298000B307F70023A007006F00C0018327C10130
:1029900093871700232EF1000327C10193077000CE
:1029A000E3F8E7FA1300000013010102678000005A
:1029B000130101FD232611022326A1002324B100C7
:1029C0002322C1008327C100232EF100EF20C0780D
:1029D0008327C10103A747049307F0FF6316F7009D
:1029E0008327C10123A207048327C10103A787040A
:1029F0009307F0FF6316F7008327C10123A40704A0
:102A0000EF2080798327C10183A78703639E070096
:102A10008327C10193874702032641008325810054
:102A200013850700EF10007F0325C101EFF05F8DD4
:102A3000130000008320C10213010103678000001E
:102A4000130101FC232E1102232EA100232CB1001F
:102A50002328D1002326E1002324F10023220101B1
:102A60002320110193070600231BF1008327C101D6
:102A700063960700737004306F0000000327C100E5
:102A80009307900063F6E700737004306F00000056
:102A9000835761018325410013850700EF10D07E25
:102AA0002324A102832781026386071C83278102D6
:102AB00003A7070383566101B70700409387F7FF19
:102AC000B387F60093972700B307F7002322F1029C
:102AD0008327410293F7C7FF2322F1028327410294
:102AE00093F7370063860700737004306F000000AF
:102AF0008357610113870700832601000326C10065
:102B00008325810103258102EF1050410326010135
:102B10008325C10103254102EFD0DFC01307050063
:102B20008327810223A0E7008327810063880700B1
:102B3000832781000327810223A0E700EF20C061E3
:102B400097E70100938707AF83A707001387170054
:102B500097E70100938707AE23A0E70097E70100FE
:102B60009387478683A707006398070297E70100CA
:102B7000938747850327810223A0E70097E7010099
:102B8000938747AB03A70700930710006312F7046E
:102B9000EF10904B6F00C00397E70100938747AA9F
:102BA00083A707006396070297E701009387878151
:102BB00083A7070083A7C7020327C100636AF70042
:102BC00097E70100938707800327810223A0E7008E
:102BD00097E701009387C7A783A70700138717000C
:102BE00097E701009387C7A623A0E70097E70100B6
:102BF000938707A603A707008327810223A4E7047E
:102C00008327810203A7C70297E70100938707A3E1
:102C100083A7070063FCE7008327810203A7C7029D
:102C200097E70100938787A123A0E700832781020C
:102C300003A7C7029307070093972700B387E7000E
:102C40009397270017E701001307478B3387E700A7
:102C500083278102938747009385070013050700A8
:102C6000EFE08FB4930710002326F102EF20C0524B
:102C70006F00C0009307F0FF2326F1020327C10273
:102C8000930710006318F70297E701009387479BAB
:102C900083A707006380070297D701009387877295
:102CA00083A7070083A7C7020327C10063F4E700D7
:102CB000EFD01F8E8327C102138507008320C10335
:102CC0001301010467800000130101FD2326110296
:102CD0002326A100EF2040488327C100639A070004
:102CE00097D701009387076E83A707006F008000C6
:102CF0008327C100232EF1008327C101938747005A
:102D000013850700EFE08FBE8327C10183A78702E9
:102D1000638A07008327C101938787011385070012
:102D2000EFE0CFBC8327C10193874700938507005D
:102D300017E501001305458DEFE00FA797E70100A8
:102D40009387C78D83A707001387170097E70100B4
:102D50009387C78C23A0E70097E701009387478FED
:102D600083A707001387170097E701009387478E13
:102D700023A0E700EF20404297E701009387478CAC
:102D800083A707006382070497D7010093878763AF
:102D900083A707000327C1016312F70297E7010029
:102DA0009387878B83A707006386070073700430BF
:102DB0006F000000EFD0CFFD6F000001EF20C039A1
:102DC000EF208001EF20403D130000008320C1026E
:102DD0001301010367800000130101FD2326110286
:102DE0002326A1002324B100232E01008327C10044
:102DF00063960700737004306F0000008327810022
:102E000063960700737004306F00000097E70100BD
:102E10009387878483A70700638607007370043055
:102E20006F000000EF00101D97E701009387C78037
:102E300083A70700232CF1008327C10083A7070085
:102E400003278100B307F700232AF1008327C1007D
:102E500083A70700032781016376F7028327C10058
:102E600083A70700032741016370F704032741018B
:102E70008327810163FAE70293071000232EF100F4
:102E80006F0080028327C10083A707000327410149
:102E90006368F700032741018327810163F6E70098
:102EA00093071000232EF1008327C100032741015F
:102EB00023A0E7008327C1016382070297D701009F
:102EC0009387475083A70700938747001385070020
:102ED000EFE0CFA103254101EF10502FEF00D013F9
:102EE0002328A1008327010163940700EFD04FEA54
:102EF000130000008320C10213010103678000005A
:102F0000130101FD232611022326A100232E010017
:102F10008327C1006380070697D701009387C77393
:102F200083A7070063860700737004306F000000FA
:102F3000EF00500C97D701009387077083A7070015
:102F40000327C100B307F700232CF10097D7010036
:102F50009387474783A70700938747001385070098
:102F6000EFE0CF9803258101EF105026EF00D00A43
:102F7000232EA1008327C10163940700EFD04FE106
:102F8000130000008320C1021301010367800000C9
:102F9000130101FD232611022326A1008327C1006E
:102FA000232CF1008327810163960700737004309E
:102FB0006F00000097D701009387C74083A70700E1
:102FC000032781016316F700232E01006F00400ADA
:102FD000EF2080188327810183A74701232AF1006E
:102FE000EF20801B97D701009387476083A70700D6
:102FF00003274101630CF70097D701009387475FD0
:1030000083A70700032741016318F70093072000F7
:10301000232EF1006F00C0050327410197D701005F
:10302000938707606314F7028327810183A78702D0
:103030006398070093073000232EF1006F004003D0
:1030400093072000232EF1006F0080020327410127
:1030500097D701009387475B6318F70093074000F9
:10306000232EF1006F00C00093071000232EF10003
:103070008327C101138507008320C10213010103C7
:1030800067800000130101FD232611022326A10001
:10309000EF20800C8327C100639A070097D70100B7
:1030A0009387473283A707006F0080008327C10002
:1030B000232EF1008327C10183A7C702232CF1002F
:1030C000EF20800D83278101138507008320C10233
:1030D0001301010367800000130101FD2326110283
:1030E0002326A100EFD00FE293070500232EF10065
:1030F0008327C100639A070097D701009387872C25
:1031000083A707006F0080008327C100232CF100F4
:103110008327810183A7C702232AF1008327C101E6
:1031200013850700EFD04FDC83274101138507008B
:103130008320C1021301010367800000130101FD18
:10314000232611022326A1002324B100232E0100EF
:10315000032781009307900063F6E7007370043043
:103160006F000000032781009307900063F6E700DB
:10317000930790002324F100EF10107E8327C100F5
:10318000639A070097D701009387C72383A7070097
:103190006F0080008327C100232CF1008327810169
:1031A00083A70705232AF100032741018327810014
:1031B000630EF716032781008327410163FEE702B0
:1031C00097D701009387072083A707000327810172
:1031D0006302F70497D701009387C71E83A70700F0
:1031E00083A7C702032781006366F70293071000D5
:1031F000232EF1006F00000297D701009387871CF0
:1032000083A70700032781016316F70093071000C7
:10321000232EF1008327810183A7C7022328F10011
:103220008327810103A707058327810183A7C7029D
:103230006318F700832781010327810023A6E70293
:10324000832781010327810023A8E70483278101C5
:1032500083A7870163CC07001307A00083278100A1
:103260003307F7408327810123ACE70083278101DF
:1032700083A64701032701019307070093972700BF
:10328000B387E7009397270017D701001307072795
:10329000B387E7006396F600930710006F00800085
:1032A00093070000638C07068327810193874700FB
:1032B00013850700EFD09FE38327810103A7C7028F
:1032C00097D701009387873783A7070063FCE70040
:1032D0008327810103A7C70297D701009387073689
:1032E00023A0E7008327810103A7C70293070700F4
:1032F00093972700B387E7009397270017D701001C
:103300001307C71F3387E70083278101938747008F
:103310009385070013050700EFD01FC90327C101DC
:10332000930710006314F700EFD08FA6EF10D0665C
:10333000130000008320C102130101036780000015
:10334000130101FD232611022326A100EF10D060F6
:103350008327C100639A070097D7010093878706E8
:1033600083A707006F0080008327C100232EF10090
:103370008327C1019387470013850700EFD01FD72C
:103380008327C10183A78702638A07008327C101BE
:103390009387870113850700EFD05FD58327C1018D
:1033A000938747009385070017D50100130545272C
:1033B000EFD09FBFEF10505E97D701009387870033
:1033C00083A707000327C1016314F70697D70100FD
:1033D0009387072783A707006382070297D7010017
:1033E0009387872783A707006386070073700430DD
:1033F0006F000000EFD0CF996F00400597D7010014
:103400009387072203A7070097D701009387872296
:1034100083A70700631AF70097D70100938787FAFD
:1034200023A007006F008002EF0090286F000002C9
:1034300097D701009387C72083A7070063880700F9
:10344000EF109051EF105019EF10105513000000BD
:103450008320C1021301010367800000130101FEF4
:103460002326A100232E01008327C100232CF10075
:103470008327C10063960700737004306F0000005B
:103480008327810103A7470197D701009387471935
:103490006316F700930710006F0080009307000089
:1034A000638E07028327810103A7870297D7010054
:1034B000938747146304F7028327810183A7870258
:1034C00063960700930710006F00800093070000C9
:1034D0006386070093071000232EF1008327C101A4
:1034E000138507001301010267800000130101FD2D
:1034F000232611022326A1008327C100232EF100D9
:103500008327C10063960700737004306F000000CA
:103510008327C1016384070C97D70100938787EA4B
:1035200083A707000327C101630AF70AEF10D042FF
:103530000325C101EFF09FF2130705009307100068
:10354000631CF7088327C101938747001385070091
:10355000EFD0DFB98327C10103A7C70297D70100C6
:103560009387C70D83A7070063FCE7008327C1018A
:1035700003A7C70297D701009387470C23A0E70052
:103580008327C10103A7C70293070700939727006A
:10359000B387E7009397270017D70100130707F6B3
:1035A0003387E7008327C10193874700938507008E
:1035B00013050700EFD05F9F8327C10103A7C70250
:1035C00097D70100938707E083A7070083A7C70267
:1035D0006364F700EFC0DFFBEF10103C1300000046
:1035E0008320C1021301010367800000130101FD64
:1035F000232611022326A100232E01008327C100C8
:10360000232CF1008327C1006396070073700430F8
:103610006F000000EFD00F8F93070500232AF10001
:1036200003258101EFF09FE31307050093071000C6
:103630006314F70C97D701009387070283A707004D
:103640006390070A8327810103A7C70297D7010068
:10365000938747D783A7070083A7C7026366F7004E
:1036600093071000232EF1008327810193874700E1
:1036700013850700EFD09FA78327810103A7C70207
:1036800097D70100938787FB83A7070063FCE700B8
:103690008327810103A7C70297D70100938707FA01
:1036A00023A0E7008327810103A7C7029307070030
:1036B00093972700B387E7009397270017D7010058
:1036C0001307C7E33387E700832781019387470008
:1036D0009385070013050700EFD01F8D6F00C00111
:1036E00083278101938787019385070017D5010000
:1036F000130545F0EFD05F8B832741011385070049
:10370000EFC09FFE8327C101138507008320C102FC
:103710001301010367800000130101FE232E110035
:10372000930800001308000093070000130700002F
:10373000930600001306004097D501009385858C01
:1037400017150000130505FBEFF08FAF2326A1002E
:103750000327C100930710006316F700EF20C03A5B
:103760002326A1000327C10093071000631EF70260
:103770007370043097D701009387C7ED1307F0FFEC
:1037800023A0E70097D70100938787EB130710006A
:1037900023A0E70097D70100938707EA23A007003B
:1037A000EFC05FC46F0040018327C100639607002C
:1037B000737004306F000000130000008320C1010B
:1037C0001301010267800000130101FF232611008D
:1037D0007370043097D70100938787E623A0070012
:1037E000EFC09FD2130000008320C100130101012C
:1037F0006780000097D70100938707E683A707003B
:103800001387170097D70100938707E523A0E700E8
:103810001300000067800000130101FE232E110039
:103820002326010097D70100938707E383A70700AA
:1038300063960700737004306F000000EF10D01122
:1038400097D70100938747E183A707001387F7FF06
:1038500097D70100938747E023A0E70097D701009F
:10386000938787DF83A707006394071697D7010024
:10387000938747DC83A70700638C07146F00800CD5
:1038800097D70100938707D783A7C70083A7C700EF
:103890002324F10083278100938787011385070084
:1038A000EFD0DF84832781009387470013850700CB
:1038B000EFD0DF838327810003A7C70297D70100DA
:1038C0009387C7D783A7070063FCE700832781009E
:1038D00003A7C70297D70100938747D623A0E70025
:1038E0008327810003A7C702930707009397270048
:1038F000B387E7009397270017D70100130707C086
:103900003387E7008327810093874700938507006B
:1039100013050700EFD04FE98327810003A7C702F3
:1039200097D70100938707AA83A7070083A7C70239
:10393000636AF70097D70100938707D11307100038
:1039400023A0E70097D701009387C7CA83A7070082
:10395000E39807F297D701009387C7CE83A70700A4
:10396000638807046F00C003EF00002B9307050076
:10397000638A070097D70100938707CD13071000CC
:1039800023A0E70097D701009387C7CB83A7070041
:103990001387F7FF97D701009387C7CA23A0E700D3
:1039A00097D70100938707CA83A70700E39E07FA0A
:1039B00097D70100938747C903A707009307100013
:1039C0006318F700930710002326F100EFC05FBCD7
:1039D000EF10807C8327C100138507008320C1017D
:1039E0001301010267800000130101FE232E110064
:1039F000EF10807697D70100938707C483A707004D
:103A00002326F100EF1040798327C10013850700BA
:103A10008320C1011301010267800000130101FE30
:103A2000232E1100EFC01FCE930705002326F100BF
:103A300097D70100938747C083A707002324F1008D
:103A40008327C10013850700EFC01FCA83278100A9
:103A5000138507008320C101130101026780000064
:103A600097D70100938707BD83A707001385070039
:103A700067800000130101FD232611022326A10007
:103A80002324B1002322C100232E01009307A000AC
:103A9000232CF100EFF01FD697D70100938787B949
:103AA00083A7070003278100636CF7148327810134
:103AB0009387F7FF232CF1008327C10193975700C9
:103AC0000327C100B306F70003278101930707000E
:103AD00093972700B387E7009397270017D7010034
:103AE0001307C7A1B387E7001306100093850700EB
:103AF00013850600EF108004130705008327C1011A
:103B0000B387E700232EF10083278101E39007FAB2
:103B10008327C101939757000327C1003307F7009C
:103B200097D70100938787AC83A70700130620006F
:103B30009385070013050700EF10400013070500E9
:103B40008327C101B387E700232EF1008327C1013A
:103B5000939757000327C1003307F70097D7010059
:103B6000938707A983A70700130620009385070002
:103B700013050700EF00907C130705008327C101A0
:103B8000B387E700232EF1008327C10193975700E5
:103B90000327C100B307F7001306400097D50100C3
:103BA000938585A613850700EF005079130705005C
:103BB0008327C101B387E700232EF1008327C101CA
:103BC000939757000327C100B307F700130630008F
:103BD00097D501009385C5A413850700EF001076E3
:103BE000130705008327C101B387E700232EF100E7
:103BF00083274100638607008327410023A0070035
:103C0000EFF09FC18327C101138507008320C10204
:103C10001301010367800000130101FD2326110237
:103C2000232E010097D70100938707A383A70700DE
:103C3000639C072297D70100938707A083A70700FB
:103C40001387170097D701009387079F23A0E700EA
:103C500097D701009387479E83A70700232CF10085
:103C600083278101639C070697D7010093870798F4
:103C700083A7070083A707006386070073700430DB
:103C80006F00000097D701009387479683A707002E
:103C9000232AF10097D701009387879503A7070090
:103CA00097D701009387879423A0E70097D7010057
:103CB000938707940327410123A0E70097D70100CA
:103CC0009387C79883A707001387170097D701002A
:103CD0009387C79723A0E700EF10001097D7010044
:103CE0009387479783A7070003278101636CF71227
:103CF00097D701009387878F83A7070083A70700C3
:103D000063960700930710006F0080009307000080
:103D1000638C070097D701009387C7931307F0FFC1
:103D200023A0E7006F00001097D701009387078C4E
:103D300083A7070083A7C70083A7C7002328F10034
:103D40008327010183A747002326F1000327810170
:103D50008327C100637CF70097D701009387878F83
:103D60000327C10023A0E7006F00C00B83270101D8
:103D70009387470013850700EFD04FB783270101D2
:103D800083A78702638A070083270101938787013E
:103D900013850700EFD08FB58327010103A7C70262
:103DA00097D701009387878983A7070063FCE70003
:103DB0008327010103A7C70297D7010093870788CC
:103DC00023A0E7008327010103A7C7029307070089
:103DD00093972700B387E7009397270017C7010041
:103DE0001307C7713387E7008327010193874700D3
:103DF0009385070013050700EFD00F9B8327010170
:103E000003A7C70297C701009387C75B83A7070073
:103E100083A7C702E36EF7EC93071000232EF1008F
:103E20006FF01FED97C701009387C75983A707005D
:103E300003A7C70297C601009386466C9307070045
:103E400093972700B387E70093972700B387F6007F
:103E500003A707009307100063F6E702930710001B
:103E6000232EF1006F00000297C701009387877D22
:103E700083A707001387170097C701009387877CE4
:103E800023A0E70097C701009387077C83A707005B
:103E90006386070093071000232EF1008327C101DA
:103EA000138507008320C10213010103678000000E
:103EB000130101FE232E110097C701009387C779D4
:103EC00083A70700638C070097C701009387C77714
:103ED0001307100023A0E7006F00C01897C7010068
:103EE0009387877623A0070097C701009387874DA4
:103EF00083A7070083A707032326F100B7A7A5A57B
:103F00009387575A2324F1008327C10083A7070012
:103F1000032781006310F7048327C10093874700BC
:103F200083A70700032781006316F7028327C100D8
:103F30009387870083A7070003278100631CF7008E
:103F40008327C1009387C70083A707000327810049
:103F50006302F70697C701009387C74603A70700C8
:103F600097C701009387074683A7070093874703F6
:103F70009385070013050700EF40C0186F0080030A
:103F800097C701009387876B83A707006396070095
:103F9000737004306F00000097C701009387076AB1
:103FA00083A707001387F7FF97C701009387076967
:103FB00023A0E70097C701009387476803A707007E
:103FC00097C60100938686539307070093972700AF
:103FD000B387E70093972700B387F60083A707000E
:103FE000E38007FA97C701009387476503A7070097
:103FF0009307070093972700B387E700939727005D
:1040000017C701001307874FB387E7002322F1008A
:104010008327410083A7470003A747008327410068
:1040200023A2E7008327410003A74700832741001D
:1040300093878700631CF7008327410083A747000D
:1040400003A747008327410023A2E70083274100FD
:1040500083A7470003A7C70097C701009387873648
:1040600023A0E700130000008320C1011301010217
:1040700067800000130101FD232611022326A10001
:104080002324B1008327C1006396070073700430B6
:104090006F00000097C701009387C73283A707000E
:1040A00093878701938507000325C100EFC09FF721
:1040B00097C701009387073183A7070093874700BD
:1040C00013850700EFD08F82032781009307F0FF4D
:1040D0006314F70297C701009387C72E83A70700D1
:1040E000938747009385070017C5010013054553C3
:1040F000EFC09FEB6F00400297C701009387C75343
:1041000083A7070003278100B307F700232EF100E0
:104110000325C101EF00900B130000008320C102B2
:104120001301010367800000130101FD2326110222
:104130002326A1002324B1002322C1008327C1002C
:1041400063960700737004306F00000097C701008A
:104150009387875083A70700639607007370043026
:104160006F00000097C701009387C72583A707004A
:10417000832681003707008033E7E60023ACE700A1
:1041800097C701009387072483A7070093878701B8
:10419000938507000325C100EFC01FE197C7010009
:1041A0009387472283A7070093874700138507005B
:1041B000EFC0DFF3032741009307F0FF6314F7021A
:1041C00097C701009387072083A7070093874700BD
:1041D0009385070017C5010013058544EFC0DFDC98
:1041E0006F00400297C701009387074583A7070028
:1041F00003274100B307F700232EF1000325C10177
:10420000EF00C07C130000008320C10213010103F2
:1042100067800000130101FD232611022326A1005F
:104220002324B1002322C1008327C1006396070025
:10423000737004306F00000097C7010093878718E0
:1042400083A7070093878701938507000325C10093
:10425000EFC09FD597C701009387C71683A70700B4
:104260009387470013850700EFC05FE803274100ED
:10427000930710006314F70297C701009387871410
:1042800083A70700938747009385070017C50100A0
:1042900013050539EFC05FD16F00400297C70100D9
:1042A0009387873983A7070003278100B307F700A7
:1042B000232EF1000325C101EF004071130000001F
:1042C0008320C1021301010367800000130101FD77
:1042D000232611022326A1008327C10083A7C7003C
:1042E00083A7C700232CF100832781016396070071
:1042F000737004306F00000083278101938787016A
:1043000013850700EFC09FDE97C701009387C7346E
:1043100083A70700639E07068327810193874700D1
:1043200013850700EFC09FDC8327810103A7C70225
:1043300097C701009387873083A7070063FCE700D6
:104340008327810103A7C70297C701009387072F1F
:1043500023A0E7008327810103A7C7029307070073
:1043600093972700B387E7009397270017C70100AB
:104370001307C7183387E700832781019387470016
:104380009385070013050700EFC01FC26F00C0012F
:1043900083278101938787019385070017C5010053
:1043A00013054525EFC05FC08327810103A7C7021E
:1043B00097C701009387070183A7070083A7C70258
:1043C00063F0E70293071000232EF10097C7010066
:1043D000938787271307100023A0E7006F00800052
:1043E000232E01008327C101138507008320C1020A
:1043F0001301010367800000130101FD2326110250
:104400002326A1002324B10097C701009387C72466
:1044100083A7070063960700737004306F000000E5
:1044200003278100B70700803367F7008327C100A7
:1044300023A0E7008327C10083A7C700232CF10036
:104440008327810163960700737004306F000000BA
:104450000325C100EFC09FC98327810193874700CF
:1044600013850700EFC09FC88327810103A7C702F8
:1044700097C701009387871C83A7070063FCE700A9
:104480008327810103A7C70297C701009387071BF2
:1044900023A0E7008327810103A7C7029307070032
:1044A00093972700B387E7009397270017C701006A
:1044B0001307C7043387E7008327810193874700E9
:1044C0009385070013050700EFC01FAE8327810106
:1044D00003A7C70297C701009387C7EE83A707000A
:1044E00083A7C70263F0E70293071000232EF100B1
:1044F00097C70100938747151307100023A0E70013
:104500006F008000232E01008327C101138507005F
:104510008320C1021301010367800000130101FF22
:104520002326A1008327C10063960700737004301F
:104530006F00000097C701009387471103A707008A
:104540008327C10023A0E70097C701009387C70E08
:1045500003A707008327C10023A2E7001300000080
:104560001301010167800000130101FD23261102E0
:104570002326A1002324B1008327C10063960700EE
:10458000737004306F00000083278100639607007A
:10459000737004306F000000EF00103C97C70100FB
:1045A0009387870983A70700232CF10083278100C5
:1045B00003A707009307F0FF6316F700232E0100FF
:1045C0006F0000098327C10003A7070097C70100F8
:1045D0009387C70783A707006300F7028327C100FB
:1045E00083A74700032781016368F7009307100042
:1045F000232EF1006F00C0058327C10083A7470069
:10460000032781013307F7408327810083A7070031
:10461000637CF7028327810003A707008327C1007B
:1046200083A6470083278101B387F6403307F7004D
:104630008327810023A0E7000325C100EFF01FEED0
:10464000232E01006F00C00093071000232EF100FD
:10465000EF0090348327C101138507008320C10236
:10466000130101036780000097C701009387C7FD0E
:104670001307100023A0E70013000000678000006C
:10468000130101FE2326A1008327C100638E0700CA
:104690008327C100232CF1008327810183A7C7044E
:1046A000232EF1006F008000232E01008327C1011B
:1046B000138507001301010267800000130101FE4A
:1046C0002326A1002324B1008327C100638C0700A7
:1046D0008327C100232EF1008327C1010327810016
:1046E00023A6E70413000000130101026780000005
:1046F000130101FE232E11002326A100EF0000214B
:1047000097C70100938787DF03A70700930710006F
:10471000E3F6E7FEEFB0DFE76FF05FFE130101FCA9
:10472000232E1102232EA100232CB100232AC10025
:104730002328D100930707002317F1002326010245
:104740006F004004032781018327C102B307F700EC
:1047500003C707008326C1018327C102B387F60080
:10476000238AE702032781018327C102B307F700E9
:1047700083C70700638007028327C102938717005E
:104780002326F1020327C1029307F000E3FCE7FAB6
:104790006F008000130000008327C101A38107047C
:1047A000032741019307900063F6E7009307900009
:1047B000232AF1008327C1010327410123A6E70231
:1047C0008327C1010327410123A8E7048327C101EF
:1047D00023AA07048327C101938747001385070095
:1047E000EFC0CFFA8327C1019387870113850700A4
:1047F000EFC0CFF98327C1010327C10123A8E70038
:104800001307A000832741013307F7408327C10125
:1048100023ACE7008327C1010327C10123A2E702DC
:104820008327C10123A207048327C10123AC070406
:104830008327C10123AE0704130000008320C103B6
:104840001301010467800000130101FE232E1100F3
:10485000232601006F0080030327C1009307070090
:1048600093972700B387E7009397270017C70100A6
:104870001307C7C8B387E70013850700EFC08FEBA6
:104880008327C100938717002326F1000327C10067
:1048900093079000E3F2E7FC17C50100130585D2EA
:1048A000EFC04FE917C50100130505D3EFC08FE82E
:1048B00017C50100130505D4EFC0CFE717C50100E8
:1048C000130585D4EFC00FE717C50100130545D5C3
:1048D000EFC04FE697C70100938747D117C7010084
:1048E000130747CE23A0E70097C70100938747D05F
:1048F00017C70100130747CE23A0E70013000000ED
:104900008320C1011301010267800000130101FE31
:10491000232E11006F008009EFE0DFED97C7010043
:10492000938787CE83A7070093B7170093F7F70FF6
:104930002326F100EFE05FEE8327C10063980706AE
:10494000EF00900197C70100938707CC83A7C700AA
:1049500083A7C7002324F1008327810093874700A2
:1049600013850700EFC08FF897C70100938787CCA6
:1049700083A707001387F7FF97C70100938787CBAB
:1049800023A0E70097C70100938747C983A70700C3
:104990001387F7FF97C70100938747C823A0E70055
:1049A000EF00807F03258100EF00C03F97C7010023
:1049B0009387C7C683A70700E39007F6130000009C
:1049C0008320C1011301010267800000130101FE71
:1049D000232E11002326A10097C701009387879EED
:1049E00083A707000327C10023A2E70097C70100A0
:1049F000938787C483A707000327C1006378F70262
:104A000097C701009387C7BE03A7070097C7010098
:104A10009387479B83A707009387470093850700E9
:104A200013050700EFC00FE06F00000597C70100F6
:104A30009387C7BB03A7070097C701009387879891
:104A400083A7070093874700938507001305070096
:104A5000EFC04FDD97C701009387C7BF83A707004B
:104A60000327C100637AF70097C70100938787BEC9
:104A70000327C10023A0E700130000008320C10129
:104A80001301010267800000130101FD23261102BA
:104A9000930705002324B1002317F1008327810029
:104AA000639E07008357E100939727001385070053
:104AB000EF20C02E930705006F0080008327810040
:104AC000232CF10083278101638A07021305000666
:104AD000EF20C02C232EA1008327C101638A070089
:104AE0008327C1010327810123A8E7026F0040014A
:104AF00003258101EF20404A6F008000232E010032
:104B00008327C101638207028327C10103A707032B
:104B10008357E10093972700138607009305500AF7
:104B200013050700EF20006A8327C10113850700E2
:104B30008320C1021301010367800000130101FCFF
:104B4000232E1102232C81022326A1002324B1004D
:104B50002322C100232601028327810083A70700A7
:104B60006388071C832781002324F10283278102A5
:104B700083A7470003A747008327810223A2E700FA
:104B80008327810203A74700832781029387870039
:104B9000631CF7008327810283A7470003A7470010
:104BA0008327810223A2E7008327810283A747008E
:104BB00083A7C7002322F102832781002320F1026B
:104BC0008327010283A7470003A747008327010229
:104BD00023A2E7008327010203A7470083270102DE
:104BE00093878700631CF7008327010283A7470090
:104BF00003A747008327010223A2E70083270102BE
:104C000083A7470083A7C700232EF1008327C10293
:104C1000939757000327C100B307F7000327C1018B
:104C200023A0E7008327C102939757000327C10001
:104C3000B307F7000327C1011307470323A2E700C7
:104C40008327C102939757000327C100B307F700DA
:104C50000327C1010327870423A4E7008327C10298
:104C6000939757000327C100B307F70003274100BC
:104C700023A6E7008327C102939757000327C100AB
:104C8000B307F7000327C1010327C70223A8E700E2
:104C900003274100930730006314F7028327C10103
:104CA00083A78702638E07008327C102939757006B
:104CB0000327C100B307F7001307200023A6E7006E
:104CC0008327C102939757000327C100B307F7005A
:104CD0000327C1010327070523AAE7008327C10291
:104CE000939757000327C100B307F70023AC0700D1
:104CF0008327C10183A607038327C1029397570027
:104D00000327C1003304F70013850600EF00C0033A
:104D100093070500231EF4008327C1029387170021
:104D20002326F1020327C10183274102E316F7E896
:104D30008327C102138507008320C1030324810355
:104D40001301010467800000130101FE2326A10066
:104D5000232E01006F00C0018327C1009387170035
:104D60002326F1008327C10193871700232EF1002A
:104D70008327C10003C707009307500AE30EF7FC1F
:104D80008327C10193D72700232EF1008327C10178
:104D90009397070193D707011385070013010102B9
:104DA00067800000130101FE232E11002326A100BD
:104DB0008327C10083A7070313850700EF20C01DC9
:104DC0000325C100EF20401D130000008320C10116
:104DD0001301010267800000130101FF97C7010062
:104DE0009387C78083A7070083A707006396070000
:104DF000930710006F00800093070000638C07008A
:104E000097C70100938707851307F0FF23A0E700EA
:104E10006F00000397B701009387477D83A70700C2
:104E200083A7C70083A7C7002326F1008327C100FB
:104E300003A7470097C701009387C78123A0E70016
:104E4000130000001301010167800000130101FF3E
:104E500097B701009387075783A707002326F10020
:104E60008327C1001385070013010101678000003B
:104E7000130101FF97B701009387877C83A7070081
:104E800063980700930710002326F1006F0040028B
:104E900097B701009387477C83A7070063980700B3
:104EA000930720002326F1006F00800023260100D5
:104EB0008327C100138507001301010167800000EB
:104EC000130101FD232611022326A1008327C1001F
:104ED000232EF1008327C100638A07128327C101B3
:104EE00003A7C70297B701009387C74D83A70700A1
:104EF00083A7C702637CF7108327C10183A78701BB
:104F000063C2070297B701009387C74B83A70700C7
:104F100083A7C7021307A0003307F7408327C10107
:104F200023ACE7008327C10183A647018327C10182
:104F300003A7C7029307070093972700B387E700EB
:104F40009397270017B701001307475BB387E70064
:104F50006396F600930710006F008000930700002F
:104F6000638A07088327C1019387470013850700D9
:104F7000EFC0CF9797B701009387C74483A7070077
:104F800003A7C7028327C10123A6E7028327C10124
:104F900003A7C70297B701009387476A83A7070053
:104FA00063FCE7008327C10103A7C70297B701008D
:104FB0009387C76823A0E7008327C10103A7C7021F
:104FC0009307070093972700B387E700939727007D
:104FD00017B70100130787523387E7008327C10102
:104FE000938747009385070013050700EFB0DFFBA9
:104FF0006F00C00197B701009387C73C83A70700E4
:1050000003A7C7028327C10123A6E70213000000FC
:105010008320C1021301010367800000130101FD19
:10502000232611022326A1008327C100232CF1008F
:10503000232E01008327C1006386071097B7010064
:105040009387473883A70700032781016306F7008A
:10505000737004306F0000008327810183A7470528
:1050600063960700737004306F000000832781018E
:1050700083A747051387F7FF8327810123AAE70446
:105080008327810103A7C7028327810183A707051F
:10509000630AF70A8327810183A747056394070AF8
:1050A000832781019387470013850700EFC00F8492
:1050B0008327810103A707058327810123A6E70230
:1050C0008327810183A7C7021307A0003307F74096
:1050D0008327810123ACE7008327810103A7C7024F
:1050E00097B701009387875583A7070063FCE70004
:1050F0008327810103A7C70297B70100938707544D
:1051000023A0E7008327810103A7C70293070700B5
:1051100093972700B387E7009397270017B70100FD
:105120001307C73D3387E700832781019387470033
:105130009385070013050700EFB01FE793071000E2
:10514000232EF1008327C101138507008320C102AC
:1051500013010103678000007370043097B70100EA
:105160009387074E83A707006384070297B7010060
:105170009387472583A7070003A747041307170052
:1051800023A2E70497B701009387C72383A70700EB
:10519000130000006780000097B701009387474A1B
:1051A00083A707006384070497B7010093878721CB
:1051B00083A7070083A74704638A070297B7010004
:1051C0009387472083A7070003A747041307F7FF28
:1051D00023A2E70497B701009387C71E83A70700A0
:1051E00083A7470463940700736004301300000032
:1051F00067800000130101FF97B701009387871CA8
:1052000083A7070083A787012326F10097B7010032
:105210009387471B83A7070003A7C70297B701001F
:105220009387471A83A707009306A0003387E640B9
:1052300023ACE7008327C100138507001301010198
:105240006780000097B701009387C71783A70700FF
:10525000638E070097B701009387C71683A70700DF
:1052600003A747051307170023AAE70497B7010010
:105270009387471583A70700138507006780000001
:10528000130101FD232611022326A1002324B100CE
:10529000EFF09FEC97B701009387C71283A7070031
:1052A00083A787056396070897B70100938787113F
:1052B00083A707001307100023AEE70483278100AC
:1052C0006388070697B701009387C70F83A7070076
:1052D0009387470013850700EFB05FE10327810044
:1052E0009307F0FF6314F70297B701009387870DC8
:1052F00083A70700938747009385070017B5010030
:1053000013050532EFB05FCA6F00400297B7010086
:105310009387873283A7070003278100B307F7002D
:10532000232EF1000325C101EFF04FEAEFB04FA6A5
:10533000EFF09FE6EFF05FE297B7010093878708F1
:1053400083A7070083A78705232CF100832781010A
:10535000638C07028327C100638C070097B70100A5
:105360009387470683A7070023AC07046F00C0019B
:1053700097B701009387070583A7070003A7870551
:105380001307F7FF23ACE70497B701009387870360
:1053900083A7070023AE0704EFF01FE083278101F6
:1053A000138507008320C1021301010367800000F9
:1053B000130101FD232611022326A1002324B1009D
:1053C0002322C1002320D100EFF01FD997B701009D
:1053D000938747FF83A7070003A7C705930720000C
:1053E0006306F70A97B701009387C7FD83A70700F5
:1053F00083A687050327C1001347F7FF33F7E600AD
:1054000023ACE70497B701009387C7FB83A7070086
:105410001307100023AEE704832701006388070603
:1054200097B70100938707FA83A707009387470080
:1054300013850700EFB09FCB032701009307F0FF10
:105440006314F70297B701009387C7F783A7070094
:10545000938747009385070017B501001305451C86
:10546000EFB09FB46F00400297B701009387C71C4D
:1054700083A7070003270100B307F700232CF100DF
:1054800003258101EFF08FD4EFB08F90EFF0DFD0E4
:10549000EFF09FCC83274100638E070097B7010090
:1054A000938747F283A7070003A787058327410057
:1054B00023A0E70097B701009387C7F083A70700F1
:1054C00003A7C705930710006316F700232E0100FA
:1054D0006F00C00297B701009387C7EE83A707004C
:1054E00083A68705032781001347F7FF33F7E600FC
:1054F00023ACE70493071000232EF10097B70100B7
:10550000938747EC83A7070023AE0704EFF0DFC8BB
:105510008327C101138507008320C1021301010302
:1055200067800000130101FD232611022326A1003C
:105530002324B1002322C1002320D10093071000AF
:10554000232EF1008327C100639607007370043097
:105550006F0000008327C100232CF100EFF0DFBFB4
:1055600083270100638A07008327810103A787053A
:105570008327010023A0E7008327810183A7C705B4
:10558000232AF100832781011307200023AEE704BB
:10559000032741009307400063ECE708832741009D
:1055A0001397270097B70100938747A6B307F70023
:1055B00003A7070097B70100938747A5B307F70034
:1055C000678007008327810103A787058327810060
:1055D0003367F7008327810123ACE7046F004005A0
:1055E0008327810183A787051387170083278101FC
:1055F00023ACE7046F00C0038327810103278100E8
:1056000023ACE7046F00C002032741019307200089
:10561000630AF700832781010327810023ACE70495
:105620006F000001232E01006F00800013000000B6
:1056300003274101930710006316F70A83278101AE
:105640009387470013850700EFB05FAA8327810186
:1056500003A7C70297B70100938747FE83A70700F8
:1056600063FCE7008327810103A7C70297B7010006
:105670009387C7FC23A0E7008327810103A7C70204
:105680009307070093972700B387E70093972700B6
:1056900017B70100130787E63387E70083278101E7
:1056A000938747009385070013050700EFB0DF8F4E
:1056B0008327810183A78702638607007370043004
:1056C0006F0000008327810103A7C70297B701007D
:1056D000938747CF83A7070083A7C70263F4E70038
:1056E000EFA01FEBEFF05FAB8327C101138507002D
:1056F0008320C1021301010367800000130101FC34
:10570000232E1102232EA100232CB100232AC10035
:105710002328D1002326E100930710002326F1025D
:105720008327C10163960700737004306F00000087
:105730008327C1012324F102EFA0DFFC93070500BA
:105740002322F10283270101638A07008327810254
:1057500003A787058327010123A0E7008327810290
:1057600083A7C7052320F1028327810213072000A6
:1057700023AEE704032741019307400063ECE708E9
:10578000832741011397270097B701009387478923
:10579000B307F70003A7070097B70100938747886F
:1057A000B307F700678007008327810203A78705F7
:1057B000832781013367F7008327810223ACE70445
:1057C0006F0040058327810283A787051387170091
:1057D0008327810223ACE7046F00C0038327810283
:1057E0000327810123ACE7046F00C00203270102F5
:1057F00093072000630AF7008327810203278101B2
:1058000023ACE7046F000001232601026F00800033
:105810001300000003270102930710006314F70E22
:105820008327810283A78702638607007370043091
:105830006F00000097B70100938707E283A7070076
:10584000639E07068327810293874700138507001D
:10585000EFB0DF898327810203A7C70297B7010052
:105860009387C7DD83A7070063FCE70083278102D6
:1058700003A7C70297B70100938747DC23A0E7007F
:105880008327810203A7C702930707009397270086
:10589000B387E7009397270017B70100130707C6E0
:1058A0003387E700832781029387470093850700AA
:1058B00013050700EFB04FEF6F00C001832781028F
:1058C000938787019385070017B50100130585D2DB
:1058D000EFB08FED8327810203A7C70297B70100BE
:1058E000938747AE83A7070083A7C70263FCE7003F
:1058F0008327C100638807008327C10013071000B6
:1059000023A0E7008327410213850700EFA0DFDD16
:105910008327C102138507008320C10313010104FB
:1059200067800000130101FD232611022326A10038
:105930002324B1008327C1006396070073700430ED
:105940006F0000008327C100232EF100EFA09FDB32
:1059500093070500232CF1008327C10183A7C70506
:10596000232AF1008327C1011307200023AEE70497
:105970008327C10183A78705138717008327C101E8
:1059800023ACE70403274101930710006314F70ECB
:105990008327C10183A787026386070073700430E1
:1059A0006F00000097B70100938707CB83A707001C
:1059B000639E07068327C10193874700138507006D
:1059C000EFB0CFF28327C10103A7C70297B7010049
:1059D0009387C7C683A7070063FCE7008327C1013D
:1059E00003A7C70297B70100938747C523A0E70025
:1059F0008327C10103A7C7029307070093972700D6
:105A0000B387E7009397270017B70100130707AF85
:105A10003387E7008327C1019387470093850700F9
:105A200013050700EFB04FD86F00C0018327C101F5
:105A3000938787019385070017B50100130585BB80
:105A4000EFB08FD68327C10103A7C70297B7010024
:105A50009387479783A7070083A7C70263FCE700E4
:105A600083278100638807008327810013071000C4
:105A700023A0E7008327810113850700EFA0DFC67D
:105A8000130000008320C10213010103678000009E
:105A9000130101FD232611022326A1008327C10043
:105AA000232CF10083278101639A070097B7010037
:105AB0009387479183A707006F00800083278101A8
:105AC000232CF100EFF04FE98327810103A7C705DD
:105AD00093072000631CF7008327810123AE07048E
:105AE00093071000232EF1006F008000232E010089
:105AF000EFF08FEA8327C101138507008320C102DD
:105B00001301010367800000130101FE232E110021
:105B100023260100EF00500B97B70100938707B7CA
:105B200083A70700638A0702930800001308000098
:105B3000930700001307200093060000130600409F
:105B400097A501009385054F170500001305852EC5
:105B5000EFC01FEF2326A1008327C1006396070033
:105B6000737004306F0000008327C10013850700A5
:105B70008320C1011301010267800000130101FCB1
:105B8000232E1102232EA100232CB100232AC100B1
:105B90002328D1002326E100832781016396070093
:105BA000232601026F0080061305C002EF10001FBC
:105BB0002326A1028327C102638A0704EF00D000D5
:105BC0008327C1020327C10123A0E7008327C10265
:105BD0000327810123ACE7008327C102032741018A
:105BE00023AEE7008327C1020327010123A0E702B8
:105BF0008327C1020327C10023A2E7028327C10232
:105C00009387470013850700EFB04FB883278101C2
:105C100063960700737004306F0000008327C10291
:105C2000138507008320C10313010104678000006E
:105C3000130101FC232E1102232EA100232CB100FD
:105C4000232AC1002328D1002326E10023260102B4
:105C50008327C10163960700737004306F00000052
:105C600097B70100938787A283A70700638C070A71
:105C7000832781012320F102832741012322F1029E
:105C80008327C1012324F1020327810193075000D8
:105C900063C6E706EFF0CF9D1307050093072000CA
:105CA0006318F70297B701009387479E83A7070001
:105CB00013070102930600000326C10093050700A5
:105CC00013850700EFB0DF972326A1026F00800540
:105CD00097B701009387879B83A7070013070102EB
:105CE00093060000130600009305070013850700C4
:105CF000EFB01F952326A1026F00C00297B70100E5
:105D00009387C79883A70700130701029306000033
:105D1000032601019305070013850700EFB05FB666
:105D20002326A1028327C102138507008320C10314
:105D30001301010467800000130101FE2326A10066
:105D40008327C100232EF1008327C100639607003B
:105D5000737004306F0000008327C10183A7070020
:105D6000138507001301010267800000130101FD84
:105D7000232611022326A1002324B10097B7010096
:105D80009387479083A7070083A7C70083A7C7000F
:105D9000232EF1008327C101938747001385070055
:105DA000EFB0CFB48327C10103A7C7019307100049
:105DB0006310F7068327C10103A787018327C1006A
:105DC000B307F7008326C1000326810093850700EF
:105DD0000325C101EF00802213070500930710007F
:105DE0006318F70213070000930600000326C100A2
:105DF000930500000325C101EFF09FE3232CA100D0
:105E00008327810163960700737004306F000000E0
:105E10008327C10183A747020325C101E78007004B
:105E2000130000008320C1021301010367800000FA
:105E3000130101FD232611022326A10093078101EE
:105E400013850700EF00800E232EA1008327810118
:105E5000938507000325C101EF00C000EF00002873
:105E60006FF0DFFD130101FD232611022326A1009F
:105E70002324B100EFD01F989307810113850700F9
:105E8000EF004011232EA1008327810163960708AC
:105E900083278100639207020327C1008327C10182
:105EA00063ECE700EFD05F978325C1010325C100B4
:105EB000EFF0DFEB6F00800683278100638007022D
:105EC00097A701009387477C83A7070083A7070054
:105ED00093B7170093F7F70F2324F10097A701005A
:105EE0009387C77A83A607000327C1008327C101D0
:105EF000B307F7400326810093850700138506004A
:105F0000EFC01FABEFD05F919307050063980700C8
:105F1000EFA00FE86F008000EFD01F90130000008B
:105F20008320C1021301010367800000130101FEF9
:105F30002326A10097A701009387C77483A70700B2
:105F400083A7070093B7170093F7F70F138707008E
:105F50008327C10023A0E7008327C10083A7070090
:105F60006390070297A701009387C77183A7070073
:105F700083A7C70083A70700232EF1006F008000CE
:105F8000232E01008327C10113850700130101029D
:105F900067800000130101FD232611022326A100C2
:105FA000EFD09FA4232EA10097A701009387476EEF
:105FB00083A707000327C101637CF700EF00C02B14
:105FC0008327C1001307100023A0E7006F00C00063
:105FD0008327C10023A0070097A701009387476B81
:105FE0000327C10123A0E7008327C1011385070010
:105FF0008320C1021301010367800000130101FD2A
:10600000232611022326A1002324B1002322C1004C
:106010002320D100232E01008327C1000327810004
:1060200023A2E7008327C1000327C10023A8E700BC
:10603000032781008327410063E6E704032741002B
:10604000832701003307F7408327C10083A7870117
:106050006368F70093071000232EF1006F00C0065D
:1060600097A701009387476203A707008327C10012
:10607000938747009385070013050700EFA09FFA59
:106080006F0080040327410083270100637EF7002F
:1060900003278100832701006368F700930710003E
:1060A000232EF1006F00400297A701009387875DC0
:1060B00003A707008327C100938747009385070044
:1060C00013050700EFA01FF68327C1011385070002
:1060D0008320C1021301010367800000130101FD49
:1060E000232611026F0080158327810063C60714E1
:1060F00083270101232EF1008327C10183A74701D4
:10610000638A07008327C10193874700138507002F
:10611000EFA0DFFD9307410013850700EFF09FE735
:10612000232CA10083278100130790006368F710D8
:106130001397270097A70100938747F0B307F7004D
:1061400003A7070097A70100938747EFB307F7005E
:10615000678007000327C1008327C10183A7870148
:10616000B307F7000327C100930607000326810148
:10617000938507000325C101EFF05FE813070500D1
:1061800093071000631CF70A8327C10183A7470206
:106190000325C101E78007008327C10103A7C701C9
:1061A00093071000631CF7080327C1008327C10170
:1061B00083A78701B307F7001307000093060000C9
:1061C00013860700930500000325C101EFF05FA6C9
:1061D000232AA100832741016392070673700430CC
:1061E0006F0000000327C1008327C10123ACE70033
:1061F0008327C10183A7870163960700737004306A
:106200006F0000008327C10103A787018327810155
:10621000B307F700832681010326810193850700D8
:106220000325C101EFF09FDD6F0040010325C1018F
:10623000EF0090566F0080001300000097A7010048
:106240009387C74483A707001307810093060000C4
:10625000130600009305070013850700EFB01F8B9E
:1062600093070500E39207E8130000008320C102B2
:106270001301010367800000130101FD23261102B1
:106280006F00C00E97A701009387C73F83A7070041
:1062900083A7C70083A70700232CF10097A701005D
:1062A0009387473E83A7070083A7C70083A7C7003C
:1062B000232AF100832741019387470013850700B4
:1062C000EFA0DFE28327410183A7470203254101B5
:1062D000E78007008327410103A7C7019307100048
:1062E0006316F7088327410183A7870103278101EC
:1062F000B307F7002328F100032701018327810159
:1063000063F0E704832741010327010123A2E7008B
:10631000832741010327410123A8E70097A7010034
:106320009387473603A707008327410193874700D8
:106330009385070013050700EFA0DFCE6F00000371
:106340001307000093060000032681019305000057
:1063500003254101EFF0DF8D2326A1008327C10033
:1063600063960700737004306F00000097A7010068
:106370009387473183A7070083A70700E39407F0BB
:1063800097A701009387073083A70700232EF1000A
:1063900097A701009387472F03A7070097A701003E
:1063A0009387472E23A0E70097A701009387C72D67
:1063B0000327C10123A0E700130000008320C102CE
:1063C0001301010367800000130101FF2326110060
:1063D000EFE09FD897A701009387472B83A707007B
:1063E0006394070A17A5010013054527EFA09FB482
:1063F00017A501001305C527EFA0DFB397A701007C
:106400009387472817A701001307472523A0E70014
:1064100097A701009387472717A701001307472570
:1064200023A0E700130600009305C00013054000F9
:10643000EFA09FE81307050097A7010093870725A2
:1064400023A0E70097A701009387472483A70700AD
:1064500063960700737004306F00000097A7010077
:106460009387C72283A707006380070297A70100CD
:106470009387C72183A7070097A50100938585BE51
:1064800013850700EFC0CFC2EFE01FD1130000005B
:106490008320C1001301010167800000130101FD89
:1064A000232611022326A1008327C100232EF100F9
:1064B0008327C10063960700737004306F000000EB
:1064C000EFE09FC98327C10183A74701B337F000DD
:1064D00093F7F70F232CF100EFE01FCC8327810106
:1064E000138507008320C1021301010367800000A8
:1064F000130101FD232611022326A1008327C100D9
:10650000232EF1008327C1006396070073700430C7
:106510006F000000EFE05FC48327C10183A707027B
:10652000232CF100EFE05FC783278101138507006B
:106530008320C1021301010367800000130101FDE4
:10654000232611022326A1002324B1008327C100A2
:10655000232EF1008327C100639607007370043077
:106560006F000000EFE05FBF8327C10103278100B8
:1065700023A0E702EFE05FC2130000008320C10206
:106580001301010367800000130101FE232E110097
:106590001305C001EF0090002326A1008327C1004E
:1065A000638E07008327C10023A007008327C10053
:1065B0009387470013850700EFA0DF978327C1006B
:1065C000138507008320C1011301010267800000C9
:1065D000130101FC232E11022326A1002324B10064
:1065E0002322C1002320D1008327C1002324F102EC
:1065F0002322010203274100B70700FFB377F7000A
:1066000063860700737004306F0000008327410029
:1066100063960700737004306F000000EFE05F8541
:106620009307050063960700832701006396070020
:10663000930710006F008000930700006396070027
:10664000737004306F000000EFD0CF9A832781026F
:1066500083A707002320F102832581000325C100C1
:10666000EF00804103270102832781003367F70091
:1066700083274100B377F70003274100631CF7022B
:106680000327010283278100B367F7002326F10265
:106690008327810203A707008327410093C7F7FFE1
:1066A0003377F7008327810223A0E700232001002E
:1066B0006F0040048327010063880702832781025B
:1066C0009386470003274100B7070005B367F7002B
:1066D000032601009385070013850600EFD0DFA491
:1066E000232601026F0000018327810283A7070090
:1066F0002326F102EFD04F92232EA1008327010021
:10670000638407088327C10163940700EF905FE863
:10671000EFE05FAE2326A1020327C102B707000204
:10672000B377F70063980704EFE01FA38327810284
:1067300083A707002326F1020327C1028327410014
:10674000B377F700032741006310F7028327810224
:1067500003A707008327410093C7F7FF3377F700AC
:106760008327810223A0E700EFE01FA39307100017
:106770002322F1020327C102B70700019387F7FF25
:10678000B377F7002326F1028327C10213850700A0
:106790008320C1031301010467800000130101FB82
:1067A00023261104232EA100232CB100232AC1008B
:1067B0002328D1002326E1008327C101232AF102E7
:1067C000232C0102232801028327C10163960700BD
:1067D000737004306F00000003278101B70700FFCA
:1067E000B377F70063860700737004306F00000012
:1067F0008327810163960700737004306F000000E7
:10680000EFE00FE793070500639607008327C100B9
:1068100063960700930710006F0080009307000045
:1068200063960700737004306F000000EFC09FFC98
:106830008327410383A707002326F10203260101D2
:10684000832581010325C102EF00404B2324A102CF
:1068500083278102638C07028327C102232EF10262
:10686000232601008327410163880708832741030A
:1068700003A707008327810193C7F7FF3377F7004A
:106880008327410323A0E7006F0000078327C1008F
:10689000639807008327C102232EF1026F00C00511
:1068A00083274101638A070003278103B70700019B
:1068B000B367F700232CF10283270101638A0700E5
:1068C00003278103B7070004B367F700232CF10205
:1068D0008327410393864700032781018327810390
:1068E000B367F7000326C1009385070013850600F0
:1068F000EFD09F83232E0102EFC01FF22322A102BB
:106900008327C10063880708832741026394070037
:10691000EF901FC8EFE01F8E232EA1020327C103B3
:10692000B7070002B377F700639C0704EFE0DF824C
:106930008327410383A70700232EF10203260101C9
:10694000832581010325C103EF00403B9307050028
:106950006384070283274101638007028327410381
:1069600003A707008327810193C7F7FF3377F70059
:106970008327410323A0E700EFE01F8223280102C1
:106980000327C103B70700019387F7FFB377F70029
:10699000232EF1028327C103138507008320C1043E
:1069A0001301010567800000130101FD2326110278
:1069B0002326A1002324B1008327C100232EF10048
:1069C0008327C10063960700737004306F000000D6
:1069D00003278100B70700FFB377F700638607003E
:1069E000737004306F000000EFE00FF78327C101E0
:1069F00083A70700232CF1008327C10103A7070009
:106A00008327810093C7F7FF3377F7008327C101FE
:106A100023A0E700EFE04FF88327810113850700EB
:106A20008320C1021301010367800000130101FDEF
:106A3000232611022326A1008327C100232EF10063
:106A4000EF905FCC93070500232CF1008327C10151
:106A500083A70700232AF1008327810113850700FC
:106A6000EF909FC883274101138507008320C1024F
:106A70001301010367800000130101FB23261104A9
:106A80002326A1002324B100232C01028327C10067
:106A90002328F102232A01028327C10063960700FD
:106AA000737004306F00000003278100B70700FFF8
:106AB000B377F70063860700737004306F0000003F
:106AC00083270103938747002326F1028327C1020E
:106AD000938787002324F102EFC0DFD18327C1020F
:106AE00083A7C700232EF1028327010303A7070012
:106AF000832781003367F7008327010323A0E70082
:106B00006F00000E8327C10383A747002322F102F1
:106B10008327C10383A707002320F102232A010250
:106B200003270102B70700FFB377F700232EF10018
:106B300003270102B70700019387F7FFB377F70038
:106B40002320F1020327C101B7070004B377F70040
:106B5000639207028327010303A70700832701022B
:106B6000B377F7006388070293071000232AF10226
:106B70006F0040028327010303A707008327010258
:106B8000B377F700032701026316F700930710009D
:106B9000232AF10283274103638007040327C101ED
:106BA000B7070001B377F700638A07000327810363
:106BB00083270102B367F700232CF1028327010327
:106BC00003A70700B7070002B367F7009385070024
:106BD0000325C103EFD05F8283274102232EF102F8
:106BE0000327C10383278102E31EF7F083270103F4
:106BF00003A707008327810393C7F7FF3377F700C5
:106C00008327010323A0E700EFC01FC183270103EF
:106C100083A70700138507008320C1041301010522
:106C200067800000130101FD232611022326A10025
:106C30008327C100232EF1008327C10193874700DA
:106C4000232CF100EFC01FBB6F004003832781019D
:106C500003A7C70083278101938787006316F70086
:106C6000737004306F0000008327810183A7C70081
:106C7000B705000213850700EFD00FF883278101C5
:106C800083A70700E39407FC0325C101EF00C03090
:106C9000EFC09FB8130000008320C102130101035D
:106CA00067800000130101FE232E11002326A1009E
:106CB0002324B100832581000325C100EFF0DFDB31
:106CC000130000008320C10113010102678000004E
:106CD000130101FE232E11002326A1002324B1005D
:106CE000832581000325C100EFF01FCC13000000B5
:106CF0008320C1011301010267800000130101FE1E
:106D00002326A1002324B1002322C100232E010049
:106D100083274100639007020327C1008327810076
:106D2000B377F7006386070293071000232EF10064
:106D30006F0000020327C10083278100B377F700AB
:106D4000032781006316F70093071000232EF1003C
:106D50008327C1011385070013010102678000002A
:106D6000130101FE2326A1008327C100232CF1007B
:106D70008327C10063960700232E01006F000001E6
:106D80008327810183A78701232EF1008327C10177
:106D9000138507001301010267800000130101FC45
:106DA000232E11022326A10023220102EFC09FA45B
:106DB000973703009387078F83A70700639C07001B
:106DC000EF00002C973703009387C78D130710003F
:106DD00023A0E7008327C100638A0702930780008E
:106DE000138707008327C100B387E7002326F1003C
:106DF0008327C10093F73700638A07008327C10008
:106E000093F7C7FF938747002326F1008327C1002C
:106E1000638207160327C100B79701009387B7FF66
:106E200063EAE714973703009387C7862324F102A8
:106E3000973703009387078683A707002326F1026D
:106E40006F0080018327C1022324F1028327C1023E
:106E500083A707002326F1028327C10283A74700E7
:106E60000327C10063F8E7008327C10283A7070057
:106E7000E39A07FC0327C102973703009387078231
:106E8000630AF70E8327810283A707001307800098
:106E9000B387E7002322F1028327C10203A707007B
:106EA0008327810223A0E7008327C10203A74700AD
:106EB0008327C100B307F74013078000131717009B
:106EC0006378F7080327C1028327C100B307F700DF
:106ED000232EF1008327C10203A747008327C100A7
:106EE0003307F7408327C10123A2E7008327C102AC
:106EF0000327C10023A2E7008327C10183A747001E
:106F0000232CF100972703009387C7782320F102F1
:106F10006F0000018327010283A707002320F102ED
:106F20008327010283A7070083A747000327810166
:106F3000E3E2E7FE8327010203A707008327C101DD
:106F400023A0E700832701020327C10123A0E70054
:106F5000979701009387474803A707008327C1023B
:106F600083A747003307F740979701009387C746E9
:106F700023A0E700EFC05F8A8327410263940700E4
:106F8000EF10401783274102138507008320C103B8
:106F90001301010467800000130101FD2326110283
:106FA0002326A1008327C100232CF1008327C100E1
:106FB0006382070A93078000B307F040032781012B
:106FC000B307F700232CF10083278101232AF10066
:106FD000EFC05F828327410183A747002328F10088
:106FE000972703009387076B232EF1006F000001A2
:106FF0008327C10183A70700232EF1008327C10146
:1070000083A7070083A7470003270101E3E2E7FE08
:107010008327C10103A707008327410123A0E700BD
:107020008327C1010327410123A0E70083274101F2
:1070300003A74700979701009387073A83A70700A4
:107040003307F700979701009387073923A0E700DC
:10705000EFC08FFC130000008320C1021301010365
:1070600067800000979701009387073783A7070081
:107070001385070067800000130000006780000090
:10708000130101FF979701009387076193F7C7FFEB
:107090002326F100972703009387C75F0327C100CA
:1070A00023A0E700972703009387C75E23A207006A
:1070B000972703009387875E379701001307C7FF61
:1070C00023A2E700972703009387475D23A00700CB
:1070D0008327C1002324F100832781003797010013
:1070E0001307C7FF23A2E7008327810017270300A8
:1070F0001307C75A23A0E700130000001301010182
:1071000067800000130101FE2326A1002324B100A3
:107110002322C10083278100232EF1008327C10091
:10712000232CF1000327C10083278100B367F700F8
:1071300093F73700639607066F00C0028327C101EB
:1071400003A707008327810123A0E700832781018C
:1071500093874700232CF1008327C10193874700C1
:10716000232EF100832741009387D7FF0327C10017
:10717000B307F70003278101E362F7FC6F004002C9
:107180000327C10193071700232EF10083278101F4
:1071900093861700232CD100034707002380E700C4
:1071A0000327C10083274100B307F70003278101AC
:1071B000E368F7FC8327C100138507001301010270
:1071C00067800000130101FE2326A1002324B100E3
:1071D0002322C1000327C10083274100B367F700C2
:1071E00093F73700639807068327810093F7F70F1B
:1071F000232AF10083274101939787000327410148
:10720000B367F700232AF100832741019397070111
:1072100003274101B367F700232AF1008327C10048
:10722000232EF1006F0080018327C10113874700DF
:10723000232EE1000327410123A0E7000327C1001B
:1072400083274100B307F7000327C101E36EF7FC72
:107250006F00C0038327C100232CF1006F00C00121
:107260008327810113871700232CE1000327810066
:107270001377F70F2380E7000327C100832741001E
:10728000B307F70003278101E36CF7FC8327C100F4
:10729000138507001301010267800000130101FE3E
:1072A0002326A1008327C100232EF1006F000001D7
:1072B0008327C10193871700232EF1008327C10183
:1072C00083C70700E39607FE0327C1018327C10098
:1072D000B307F74013850700130101026780000020
:1072E000130101FE2326A1002324B1008327C1003E
:1072F000138717002326E10083C70700A30FF100BF
:1073000083278100138717002324E10083C7070028
:10731000230FF1008347F101638807000347F10160
:107320008347E101E304F7FC0347F1018347E101EF
:10733000B307F740138507001301010267800000BF
:10734000130101FE2326A1002324B1008327C100DD
:10735000232EF1001300000003278100930717007C
:107360002324F1008327C10193861700232ED10027
:10737000034707002380E70083C70700E39E07FC5D
:107380008327C100138507001301010267800000F5
:10739000130101FE2326A100232E0100232C01004E
:1073A0006F0000018327C100938717002326F10097
:1073B0008327C10003C7070093070002E304F7FE19
:1073C0008327C10003C707009307D002630AF700B1
:1073D0008327C10003C707009307B0026312F706B3
:1073E0008327C10083C70700938737FD93B7170032
:1073F00093F7F70F232CF1008327C1009387170021
:107400002326F1006F00C0030327C1019307070083
:1074100093972700B387E70093971700232EF10077
:107420008327C100138717002326E10083C70700C5
:10743000938707FD0327C101B307F700232EF1004F
:107440008327C10083C70700E39007FC83278101DE
:10745000638807008327C101B307F0406F008000F5
:107460008327C10113850700130101026780000013
:10747000130101FE2326A100972703009387872489
:1074800083A7070093861700172703001307872396
:107490002320D7000327C1001377F70F9726030097
:1074A00093864626B387F6002380E7000327C100B2
:1074B0009307A000630CF7009727030093878720AA
:1074C00003A7070093070004631EF7049727030030
:1074D00093874723232EF1006F00C0038327C10148
:1074E00013871700232EE10003C70700B70710F02A
:1074F000938707F023A0E700972703009387871C53
:1075000083A707001387F7FF972703009387871B3D
:1075100023A0E700972703009387C71A83A70700D4
:10752000E39E07FA93070000138507001301010289
:1075300067800000130101EB23261114232481141A
:107540002322911423202115232E3113232C4113A0
:10755000232A5113232EA100232CB1002328C1007C
:10756000232AD1002326E1002324F1002322010154
:10757000232601128327C100138A0700930A000003
:10758000832701010328410113060A0093860A009C
:107590001385070093050800EF10006393070500AB
:1075A0001388050013860700930608008327C1127D
:1075B000138717002326E11213070600939727006D
:1075C00093060113B387F60023AEE7EE8327C100CD
:1075D00013840700930400008327410113870400EC
:1075E00063E8E70483274101138704006398E700F9
:1075F000832701011307040063ECE7028327C1001E
:1076000013890700930900001306090093860900F7
:107610000325010183254101EF00507D93070500FB
:10762000138805002328F100232A01016FF09FF43D
:10763000130000006F0040018327C10183258101F1
:1076400003254100E7800700832781001387F7FFA8
:107650002324E1000327C112E340F7FE6F00400539
:107660008327C1129397270013070113B307F7006D
:1076700003A7C7EF8327C11293972700930601132F
:10768000B387F60083A6C7EF9307900063F6D70091
:10769000930770056F00800093070003B387E7002E
:1076A0000327C1018325810113850700E700070037
:1076B0008327C1121387F7FF2326E112E342F0FA72
:1076C000130000008320C114032481148324411477
:1076D000032901148329C113032A8113832A411327
:1076E0001301011567800000130101FF2326A1008B
:1076F0002324B10083268100130710006356D702AC
:107700008327C10083A707009387770093F787FF3C
:10771000938687000327C1002320D70003A84700D2
:1077200083A707006F000005032781006304070299
:107730000327C10003270700130647008326C10063
:1077400023A0C600032707009307070013080000C3
:107750006F0040020327C1000327070013064700FC
:107760008326C10023A0C600032707009307070054
:107770001308000013850700930508001301010199
:1077800067800000130101FF2326A1002324B1001C
:1077900083268100130710006356D7028327C10098
:1077A00083A707009387770093F787FF9386870067
:1077B0000327C1002320D70003A8470083A70700A1
:1077C0006F00800503278100630607020327C100BD
:1077D00003270700130647008326C10023A0C60025
:1077E00003270700930707001357F7411308070003
:1077F0006F0080020327C10003270700130647001C
:107800008326C10023A0C6000327070093070700B3
:107810001357F74113080700138507009305080065
:107820001301010167800000130101FC232E1102E6
:10783000232C8102232A91022326A1002324B100B4
:107840002322C1002320D1006F0040026300043CCA
:1078500083274100938717002322F1008327C1006B
:107860008325810013050400E7800700832741007A
:1078700083C707001384070093075002E318F4FC42
:1078800083274100938717002322F10083274100BB
:107890002328F10093070002A30BF1009307F0FFE8
:1078A000232EF1009307F0FF232CF1002320010287
:1078B00083274100138717002322E10083C70700B5
:1078C000138407009307D4FD130750056360F73254
:1078D00013972700978701009387C779B307F700AD
:1078E00003A70700978701009387C778B307F700BE
:1078F000678007009307D002A30BF1006FF05FFBD6
:1079000093070003A30BF1006FF09FFA232C0100F3
:10791000032781019307070093972700B387E700A8
:1079200093971700B307F400938707FD232CF1000A
:107930008327410083C70700138407009307F002E1
:1079400063D287049307900363CE870283274100A5
:10795000938717002322F1006FF09FFB832701001C
:10796000138747002320E10083A70700232CF100A1
:107970006F0080018327C101E3DC07F2232E0100A1
:107980006FF01FF3130000008327C101E3D207F259
:1079900083278101232EF1009307F0FF232CF100B0
:1079A0006FF01FF183270102938717002320F10254
:1079B0006FF01FF083270100138747002320E100A9
:1079C00083A707000327C1008325810013850700D3
:1079D000E70007006F00402383270100138747005B
:1079E0002320E10083A4070063960400978401002C
:1079F0009384C4678327C1016350F0080347710172
:107A00009307D002630AF706832781019385070055
:107A100013850400EF00503B130705008327C101C5
:107A2000B387E740232EF1006F00400283477101C6
:107A30000327C1008325810013850700E7000700A5
:107A40008327C1019387F7FF232EF1008327C1010C
:107A5000E34EF0FC6F0040028327C10083258100C4
:107A600013050400E7800700938414008327C101F5
:107A70009387F7FF232EF10083C7040013840700C8
:107A80006300040483278101E3C807FC8327810185
:107A90009387F7FF232CF10083278101E3DE07FAA8
:107AA0006F0000028327C1008325810013050002B7
:107AB000E78007008327C1019387F7FF232EF1009A
:107AC0008327C101E340F0FE6F000014930701001B
:107AD0008325010213850700EFF0DFCA9307050035
:107AE000138805002324F102232601038327810242
:107AF0000328C1029307080063D607048327C10047
:107B0000832581001305D002E780070083258102C9
:107B10000326C1029307000013080000B386B74094
:107B20001385060033B5A7003307C840B307A74045
:107B30001387070093870600130807002324F10228
:107B4000232601039307A0002322F1026F004006C1
:107B50009307A0002322F1026F0000049307800026
:107B60002322F1026F004003930710002320F1024B
:107B70008327C1008325810013050003E7800700E8
:107B80008327C1008325810013058007E780070054
:107B9000930700012322F1029307010083250102CC
:107BA00013850700EFF05FB42324A1022326B1025E
:107BB0000327410283477101138807008327C1010E
:107BC000032681028326C102832581000325C1008B
:107BD000EFF05F966F0040038327C100832581008B
:107BE00013050400E78007006F0000028327C1002F
:107BF0008325810013055002E780070083270101D8
:107C00002322F100130000006FF05FC61300000094
:107C10008320C1030324810383244103130101044E
:107C200067800000130101FF2326A100B70710F0B1
:107C3000938707F20327C10023A0E7006F0000002D
:107C4000130101FB232611022326A100232AB102DE
:107C5000232CC102232ED1022320E1042322F1048C
:107C6000232401052326110593070105938747FE69
:107C7000232EF1008327C101938607000326C1004C
:107C80009305000017F5FFFF1305C57EEFF0DFB980
:107C900093070000138507008320C102130101052B
:107CA00067800000130101FE2326A1002324B100F8
:107CB0002322710083278100232EF1008327C10135
:107CC00083A707000327C1001377F70F2380E7007E
:107CD0008327C10183A70700138717008327C101EA
:107CE00023A0E700130000001301010267800000D9
:107CF000130101FA232E11022326A1002324B1002F
:107D00002324C1042326D1042328E104232AF104D7
:107D1000232C0105232E1105930701062322F102CE
:107D20009307410193054101170600001306C6F7AA
:107D300037F7FFFF9346F7FF37150000130505805F
:107D40003388A5003378E8001368783B23A0070147
:107D50003305A6003377E5001367773323A2E700E6
:107D600033F7D500931547013787030013073739D9
:107D700033E7E50023A4E7003377D60093164701E5
:107D8000370703001307770633E7E60023A6E7006B
:107D90000F1000008327C1002326F102930701067C
:107DA000938787FE2324F102032781029307410171
:107DB000138507009307C10093060700032681007F
:107DC00093850700EFF05FA68327C100238007009B
:107DD0008327C100138707008327C102B307F74039
:107DE000138507008320C10313010106678000008B
:107DF000130101FF370510F0130545F403250500B5
:107E00002326A100370510F0130505F4032505000E
:107E10002324A100370510F0130545F403250500C0
:107E20008328C100E398A8FC0325C10013030500C3
:107E3000930300001317030093060000032581003D
:107E40009305050013060000B3E7B6003368C700CA
:107E5000370710F0130587F4B7150000938505FA6E
:107E600013060000B386B70093880600B3B8F80085
:107E70003307C800B387E80013870700938706001D
:107E8000130807002320F50023220501130000003A
:107E90001301010167800000130101FF2326110077
:107EA000EFF01FF59307000873A0473013000000A0
:107EB0008320C1001301010167800000130101FE4E
:107EC000232E11002326A10017850100130505307C
:107ED000EFF01FD7130000008320C101130101023E
:107EE00067800000130101FE232E11002326A1004C
:107EF000178501001305052EEFF09FD41300000035
:107F00008320C1011301010267800000130101FDFC
:107F1000232611022326A100232E01006F00400119
:107F2000130000008327C10193871700232EF1005F
:107F30000327C101B717000093877738E3D2E7FE24
:107F40001785010013058529EFF09FCF6FF0DFFC47
:107F5000130101FF23261100EF00001C1300000095
:107F60008320C1001301010167800000130101FE9D
:107F7000232E110023260100EF00C0621307050025
:107F800093071000630EF700178501001305852580
:107F9000EFF01FCB8327C10093E727002326F100D2
:107FA0008327C100138507008320C101130101024B
:107FB00067800000130101FE232E1100232601001B
:107FC000EFF01FF91707000013078706930600005C
:107FD00013061000930540061785010013050522BE
:107FE000EFD0DFB92326A1008327C10063820702F7
:107FF000EFB09F9F93070500130700009306000052
:1080000013860700930510000325C100EFD05FC25F
:1080100023240100EFB04FF0930700001385070001
:108020008320C1011301010267800000130101FDDB
:10803000232611022326A100978701009387C738C2
:1080400083A7070013874706978701009387C737E1
:1080500023A0E700978701009387473783A707008E
:1080600013874706978701009387473623A0E700C9
:10807000978701009387473503A707009307F07C94
:1080800063DEE704978701009387073483A707001F
:1080900013870783978701009387073323A0E7009F
:1080A000EFF0DFEC232EA1008327C101639E0700C0
:1080B000978701009387873103A70700B717000050
:1080C0009387F77663D0E7028327C1011385070002
:1080D000EFF05FB5EFB04FEF6F000001130000004D
:1080E0006F008000130000008320C1021301010310
:1080F00067800000737004306F0000001300000000
:1081000067800000130101FF2326A1002324B10092
:10811000737004306F000000130101FE232E110064
:1081200023240100232601006F00C00A130600006B
:108130009305400013051000EF900F98930605007B
:1081400017170300130707608327C10093972700C1
:10815000B307F70023A0D7001306000093054000E3
:1081600013051000EF904F959306050017170300B5
:108170001307475E8327C10093972700B307F700D3
:1081800023A0D700171703001307C75B8327C1007D
:1081900093972700B307F70083A707001307810011
:1081A00093060000130600009305070013850700DF
:1081B000EF900FC90326C1009305100017050000BA
:1081C0001305C51BEF804FE18327C100938717007C
:1081D0002326F1000327C10093073000E3F8E7F4FA
:1081E000130000008320C101130101026780000019
:1081F000130101FE232E1100971703009387C75622
:1082000083A7070013871700971703009387C755A5
:1082100023A0E700971703009387075503A70700DC
:108220009307301F63F2E714971703009387C75330
:1082300023A00700232601006F00000A232201006B
:1082400017170300130707508327C10093972700D0
:10825000B307F70083A707009306410013078100C7
:10826000138606009305070013850700EFA08FD43F
:108270001307050093071000630CF700971703001E
:108280009387474E1307100023A0E7006F000004F8
:1082900003278100971703009387474D83A70700A3
:1082A000630AF700971703009387C74B1307100063
:1082B00023A0E70083274100638A07009717030084
:1082C0009387474A1307100023A0E7008327C100C4
:1082D000938717002326F1000327C100930730007E
:1082E000E3DEE7F4971703009387474883A7070067
:1082F00013871700971703009387474723A0E700CA
:10830000232601006F008005171703001307874419
:108310008327C10093972700B307F70083A70700BF
:108320001306000097150300938545441385070045
:10833000EFA0CFBF1307050093071000630AF700F3
:1083400097170300938707421307100023A0E70045
:108350008327C100938717002326F1000327C1005C
:1083600093073000E3D2E7FA130000008320C10135
:108370001301010267800000130101FD2326110291
:108380002326A1002324B1008327C10083D74703FC
:108390001307901D638AE70E1307901D634AF700C9
:1083A000638207021307801D6380E7086F00C01E09
:1083B0001307E01E638EE7141307F01E638AE71AA3
:1083C0006F00801D232E0100171703001307873845
:1083D0008327810093972700B307F70083A6070040
:1083E0008327810013972700971703009387473847
:1083F000B307F7001306F0FF938507001385060007
:10840000EFA00F9F93070500232EF1000327C10162
:108410009307C0FF631CF7048327C1001307801D67
:10842000239AE7026F0040171717030013078732DC
:108430008327810093972700B307F70083A60700DF
:1084400083278100139727009717030093874732EC
:10845000B307F70013060000938507001385060095
:10846000EFA00F9993070500232EF1000327C10108
:108470009307B0FF631EF7008327C1001307901D09
:10848000239AE7026F00401193071000232EF1009A
:108490000327C10193071000630AF7009717030031
:1084A0009387472C1307100023A0E700232E010019
:1084B00017170300130707298327810093972700C5
:1084C000B307F70083A607008327810013972700CF
:1084D000971703009387C729B307F7001306000017
:1084E0009385070013850600EFA04F8293070500D0
:1084F000232EF1000327C1019307C0FF631CF7047B
:108500008327C1001307E01E239AE7026F00C0080B
:10851000171703001307072383278100939727006A
:10852000B307F70083A6070083278100139727006E
:10853000971703009387C723B307F70013060000BC
:108540009385070013850600EF905FFC93070500F5
:10855000232EF1000327C1019307B0FF631EF7002C
:108560008327C1001307F01E239AE7026F00C002A1
:1085700093071000232EF1000327C1019307100079
:10858000E302F7E4971703009387C71D1307100052
:1085900023A0E7006FF01FE38320C1021301010352
:1085A00067800000971703009387C71B83A7070006
:1085B00063860700930700006F0080009307100098
:1085C0001385070067800000B305B5009307050019
:1085D0006386B70003C70700631607003385A7400B
:1085E00067800000938717006FF09FFE130101FD65
:1085F00023229102232A51012326110223248102DE
:1086000023202103232E3101232C41012328610142
:108610002326710123248101232291012320A1011A
:10862000930A050093840500639E06381304060030
:108630009309050017890100130909BD63F8C512E4
:10864000B7070100138B05006378F6101307F00FCE
:108650003337C70013173700B357E6003309F90063
:10866000834609003387E60093060002B386E6409E
:10867000638C0600B394D40033D7EA003314D600D9
:10868000336B9700B399DA00935A040193850A007B
:1086900013050B00EF00902A1309050093850A00CB
:1086A000931B040113050B00EF00D02493DB0B0197
:1086B000930405009305050013850B00EF00D020FF
:1086C0001319090193D70901B367F900138A04004C
:1086D00063FEA700B3878700138AF4FF63E887006F
:1086E00063F6A700138AE4FFB3878700B384A7402B
:1086F00093850A0013850400EF0050241309050038
:1087000093850A0013850400EF00D01E9399090198
:1087100093040500930505001319090113850B0047
:1087200093D90901EF00501AB36939011386040087
:1087300063FCA900B30934011386F4FF63E68900E2
:1087400063F4A9001386E4FF13140A013364C40020
:10875000130A00006F000013B707000113070001A0
:10876000E36CF6EE130780016FF01FEF138A06002B
:10877000631A06009305000013051000EF00901720
:1087800013040500B7070100637EF4129307F00F8E
:1087900063F48700130A8000B35744013309F900DA
:1087A000034709009306000233074701B386E640FA
:1087B00063940612B3848440130A1000135B04010F
:1087C00093050B0013850400EF00501713090500F3
:1087D00093050B0013850400931B0401EF00901117
:1087E00093DB0B01930405009305050013850B0033
:1087F000EF00900D1319090193D70901B367F90030
:10880000938A040063FEA700B3878700938AF4FF6E
:1088100063E8870063F6A700938AE4FFB3878700C5
:10882000B384A74093050B0013850400EF001011DB
:108830001309050093050B0013850400EF00900B4E
:108840009399090193040500930505001319090183
:1088500013850B0093D90901EF001007B3693901A3
:108860001386040063FCA900B30934011386F4FFE6
:1088700063E6890063F4A9001386E4FF13940A01F8
:108880003364C4001305040093050A008320C10269
:108890000324810283244102032901028329C101A7
:1088A000032A8101832A4101032B0101832BC1008B
:1088B000032C8100832C4100032D010013010103CF
:1088C00067800000B7070001130A0001E366F4ECBB
:1088D000130A80016FF05FEC3314D40033DAE40044
:1088E000B399DA0033D7EA00935A0401B394D40061
:1088F00093850A0013050A00336B9700EF001004FC
:108900001309050093850A0013050A00931B04014F
:10891000EF00407E93DB0B019304050093050500F7
:1089200013850B00EF00407A1319090113570B014F
:108930003367E900138A0400637EA70033078700CA
:10894000138AF4FF636887006376A700138AE4FF45
:1089500033078700B304A74093850A0013850400FA
:10896000EF00C07D1309050093850A0013850400FC
:10897000EF004078930405009305050013850B0074
:10898000EF00807413170B01135707011319090126
:10899000B367E9001387040063FEA700B38787006D
:1089A0001387F4FF63E8870063F6A7001387E4FFEB
:1089B000B3878700131A0A01B384A740336AEA0019
:1089C0006FF0DFDF63ECD51EB707010063F4F60438
:1089D0001307F00FB335D7009395350033D7B600A2
:1089E0009787010093874782B387E70003C7070093
:1089F000130A00023307B700330AEA4063160A027B
:108A000013041000E3E096E833B6CA0013441600DE
:108A10006FF05FE7B707000193050001E3E0F6FCA4
:108A2000930580016FF09FFBB35CE600B3964601AF
:108A3000B3ECDC0033D4E40093DB0C01B3974401C6
:108A400033D7EA0093850B0013050400336BF7005E
:108A5000B3194601EF00806E1309050093850B00E2
:108A600013050400139C0C01EF00C068135C0C019B
:108A7000930405009305050013050C00EF00C06486
:108A80001319090113570B013367E900138404001C
:108A9000637EA700330797011384F4FF636897018F
:108AA0006376A7001384E4FF33079701B304A7405C
:108AB00093850B0013850400EF004068130905003F
:108AC00093850B0013850400EF00C062930405003A
:108AD0009305050013050C00EF00005F93170B01D1
:108AE0001319090193D70701B367F900138604002E
:108AF00063FEA700B38797011386F4FF63E897012D
:108B000063F6A7001386E4FFB387970113140401EB
:108B1000B70B01003364C4001389FBFF337D2401CC
:108B200033F92901B384A7409305090013050D000B
:108B3000EF008059935C040193050900130B0500B5
:108B400013850C00EF00405893D90901130C050060
:108B50009385090013850C00EF00005713090500E9
:108B60009385090013050D00EF00005633058501BC
:108B700093570B013385A70063748501330979018D
:108B800093570501B387270163E6F402E392F4BC2F
:108B9000B70701009387F7FF3375F500131505013B
:108BA000337BFB0033964A0133056501130A00004D
:108BB000E37AA6CC1304F4FF6FF09FB9130A000008
:108BC000130400006FF01FCC130101FB2324810468
:108BD00023229104232E31032322910323261104FF
:108BE00023202105232C4103232A51032328610339
:108BF00023267103232481032320A103232EB10103
:108C0000930C050093890500130405009384050067
:108C1000639E062613090600138A0600977A010050
:108C2000938A8A5E63F4C514B70701006376F6126F
:108C30009307F00F63F4C700130A8000B35746018F
:108C4000B38AFA0003C70A0013050002330747017D
:108C5000330AE540630C0A00B395490133D7EC00B1
:108C600033194601B364B70033944C01935A090198
:108C700093850A0013850400EF00404C930905001A
:108C800093850A00131B090113850400EF00804639
:108C9000135B0B019305050013050B00EF00C042A9
:108CA0009399090193570401B3E7F90063FAA70008
:108CB000B387270163E6270163F4A700B387270181
:108CC000B384A74093850A0013850400EF00004792
:108CD0009309050093850A0013850400EF00804185
:108CE00013140401930505009399090113050B0062
:108CF00013540401EF00403D33E48900637AA4007B
:108D000033042401636624016374A4003304240142
:108D10003304A44033554401930500008320C1046B
:108D20000324810483244104032901048329C1030A
:108D3000032A8103832A4103032B0103832BC102EE
:108D4000032C8102832C4102032D0102832DC101DA
:108D50001301010567800000B7070001130A000135
:108D6000E36EF6EC130A80016FF05FED631A060004
:108D70009305000013051000EF00C037130905002C
:108D8000B7070100637AF90E9307F00F63F4270128
:108D9000130A8000B3574901B38AFA0003C70A00D7
:108DA00013050002B384294133074701330AE54024
:108DB000E30E0AEA33194901B3DAE900B395490130
:108DC00033D7EC0093540901336BB70013850A00C5
:108DD00093850400EF008036930905009385040015
:108DE000931B090113850A00EF00C03093DB0B01D0
:108DF0009305050013850B00EF00002D93990901E1
:108E000093570B01B3E7F90033944C0163FAA700C1
:108E1000B387270163E6270163F4A700B38727011F
:108E2000B38AA7409385040013850A00EF00003140
:108E3000930905009385040013850A00EF00802B39
:108E40009305050013850B00EF00002893150B0117
:108E50009399090193D50501B3E5B90063FAA5001B
:108E6000B385250163E6250163F4A500B3852501DB
:108E7000B384A5406FF09FDFB7070001130A00011C
:108E8000E36AF9F0130A80016FF0DFF0E3E8D5E858
:108E9000B707010063FCF604930BF00F33B5DB005A
:108EA0001315350033D7A600977701009387C73590
:108EB000B387E70083CB070093050002B38BAB00B9
:108EC000338B7541631E0B0263E4360163EACC0009
:108ED0003384CC40B386D94033B58C00B384A640EC
:108EE00013050400938504006FF05FE3B7070001EA
:108EF00013050001E3E8F6FA130580016FF09FFA0D
:108F0000B3966601335D7601336DDD0033D47901AC
:108F1000B395690133DC7C0193540D01336CBC00C3
:108F20001305040093850400B31A6601EF000021C5
:108F3000130A0500938504001305040033996C019E
:108F4000931C0D01EF00001B93DC0C0113040500C2
:108F50009305050013850C00EF000017131A0A0192
:108F600013570C013367EA00130A0400637EA7005D
:108F70003307A701130AF4FF6368A7016376A7000C
:108F8000130AE4FF3307A701B309A7409385040040
:108F900013850900EF00801A93850400130405006F
:108FA00013850900EF0000159305050093040500E3
:108FB00013850C00EF00401193150C0113140401EC
:108FC00093D50501B365B4001387040063FEA500C3
:108FD000B385A5011387F4FF63E8A50163F6A50037
:108FE0001387E4FFB385A501131A0A01B70C01002A
:108FF000336AEA001384FCFFB3778A0033F48A00F3
:10900000B384A54013850700930504002326F100CF
:10901000135A0A01EF00400B930905009305040061
:1090200013050A00EF00400A13DC0A01930D050046
:1090300093050C0013050A00EF0000098327C10007
:10904000130A050093050C0013850700EF00C00705
:109050003305B50113D709013307A7006374B701BE
:10906000330A9A01B70701009387F7FF9355070169
:109070003377F70013170701B3F7F900B3854501FC
:10908000B307F70063E6B400639EB400637CF900A5
:1090900033865741B3B7C700B385A541B385F540C3
:1090A00093070600B307F9403339F900B385B4409C
:1090B000B385254133947501B3D767013365F40057
:1090C000B3D565016FF09FC51306050013050000B9
:1090D00093F61500638406003305C50093D515008B
:1090E00013161600E39605FE678000006340050630
:1090F00063C6050613860500930505001305F0FFFA
:10910000630C060293061000637AB6006358C00031
:109110001316160093961600E36AB6FE13050000B8
:1091200063E6C500B385C5403365D50093D6160008
:1091300013561600E39606FE678000009382000037
:10914000EFF05FFB13850500678002003305A04048
:1091500063D80500B305B0406FF0DFF9B305B04048
:1091600093820000EFF01FF93305A04067800200F2
:109170009382000063CA0500634C0500EFF09FF77F
:109180001385050067800200B305B040E35805FE73
:109190003305A040EFF01FF63305B04067800200B2
:02000004800278
:1000000049444C45000000002456FEFFBC55FEFF4D
:10001000D855FEFFF055FEFF0056FEFFF457FEFFD9
:100020008C57FEFFA857FEFFC057FEFFD057FEFFBC
:10003000546D7220537663001C61FEFF1C61FEFF4D
:100040001C61FEFF0462FEFFAC61FEFFF461FEFF77
:100050001C61FEFF1C61FEFF0462FEFFAC61FEFF3F
:10006000546D725100000000286E756C6C29000000
:100070004078FEFF7C7BFEFF687BFEFF7C7BFEFF03
:100080007C7BFEFF7C7BFEFF7C7BFEFFEC78FEFF33
:100090007C7BFEFF7C7BFEFF8478FEFF0479FEFF05
:1000A0007C7BFEFF9078FEFF9C78FEFF9C78FEFF35
:1000B0009C78FEFF9C78FEFF9C78FEFF9C78FEFFFC
:1000C0009C78FEFF9C78FEFF9C78FEFF7C7BFEFF09
:1000D0007C7BFEFF7C7BFEFF7C7BFEFF7C7BFEFF50
:1000E0007C7BFEFF7C7BFEFF7C7BFEFF7C7BFEFF40
:1000F0007C7BFEFF7C7BFEFF7C7BFEFF7C7BFEFF30
:100100007C7BFEFF7C7BFEFF7C7BFEFF7C7BFEFF1F
:100110007C7BFEFF7C7BFEFF7C7BFEFF7C7BFEFF0F
:100120007C7BFEFF7C7BFEFF7C7BFEFF7C7BFEFFFF
:100130007C7BFEFF7C7BFEFF7C7BFEFF7C7BFEFFEF
:100140007C7BFEFF7C7BFEFF7C7BFEFF7C7BFEFFDF
:100150007C7BFEFF7C7BFEFF7C7BFEFF7C7BFEFFCF
:100160007C7BFEFF7C7BFEFF7C7BFEFF7C7BFEFFBF
:100170004479FEFF5C7AFEFF7C7BFEFF7C7BFEFF0A
:100180007C7BFEFF7C7BFEFF7C7BFEFF7C7BFEFF9F
:100190007C7BFEFF3479FEFF7C7BFEFF7C7BFEFFD9
:1001A000EC7AFEFFF87AFEFF7C7BFEFF7C7BFEFF95
:1001B0006879FEFF7C7BFEFFE07AFEFF7C7BFEFF22
:1001C0007C7BFEFF207BFEFF6D69616F750A00007E
:1001D0006D69616F75320A0068756E6772790A0021
:1001E0004572726F7220696E20787878207461731E
:1001F0006B73200D0A000000436865636B54696DE2
:1002000065720000000102020303030304040404F6
:100210000404040405050505050505050505050592
:100220000505050506060606060606060606060672
:10023000060606060606060606060606060606065E
:100240000606060607070707070707070707070742
:10025000070707070707070707070707070707072E
:10026000070707070707070707070707070707071E
:10027000070707070707070707070707070707070E
:1002800007070707080808080808080808080808F2
:1002900008080808080808080808080808080808DE
:1002A00008080808080808080808080808080808CE
:1002B00008080808080808080808080808080808BE
:1002C00008080808080808080808080808080808AE
:1002D000080808080808080808080808080808089E
:1002E000080808080808080808080808080808088E
:1002F000080808080808080808080808080808087E
:0403000008080808D9
:100304001000000000000000017A5200017C01018D
:100314001B0D02004C00000018000000CC82FEFF00
:10032400DC05000000440E307089039507810188C4
:100334000292049305940696089709980A990B9AD1
:100344000C0370020AC144C844C944D244D344D4FF
:1003540044D544D644D744D844D944DA440E00445E
:100364000B00000050000000680000005888FEFFE9
:100374000005000000440E50748802890393059917
:100384000B810192049406950796089709980A9A96
:100394000C9B0D0320010AC144C844C944D244D370
:1003A40044D444D544D644D744D844D944DA44DB6D
:0803B400440E00440B000000A0
:1003CC00AAAAAAAA08000000FC8F010009000000DC
:040000058000004037
:00000001FF
